:100000000C94550E0C94740E0C94740E0C94740E87
:100010000C94740E0C94740E0C94740E0C94740E58
:100020000C94740E0C94B5120C94740E0C94740E03
:100030000C94740E0C94740E0C94740E0C94740E38
:100040000C94740E0C94B10F0C94582E0C94282E12
:100050000C94740E0C94740E0C94740E0C94740E18
:100060000C94740E0C94740E0C94740E0C94740E08
:100070000C94740E0C94740E0C94740E0C94740EF8
:100080000C94740E0C94740E0C94740E0F299F2B08
:100090001A299F2B362936298E29D229112A612A1D
:1000A000A3299F2B9F2BF92A0A2B302B452B9F2B03
:1000B0009F2B9F2B9F2B9F2B9F2B9F2B9F2B9F2BF0
:1000C0009F2B9F2B9F2B822B842B892B562B9F2B77
:1000D000972B322E302E3100696E636F6D70617414
:1000E00069626C6520485700202025303258002076
:1000F000504300204C430045617379436F6E747226
:100100006F6C000102031718040506151107080992
:1001100016120A000B0C13100F0E0D14040E1F0EF6
:100120000E0E0E000E0E0E0E1F0E0400040E1F000B
:100130001F0E0400000404040010081300100B1329
:1001400000130B130001021900011A1900191A19E2
:10015000080C1E1F1E0C080002060F1F0F060200CF
:100160000E11111F1B1B1F001F0A0A0A0A0A1F007B
:100170001C101810160505050C17141714170C0081
:10018000040A110A0A0E00001C10181216020207B7
:100190001C101816110204071C1018161102010673
:1001A0001C1018151507010100000017151515176B
:1001B000121212121200000000000017111714177B
:1001C0001711131117000000000000151517111169
:1001D0001714171117000000070505050505050789
:1001E0000707070707070707030509121418100078
:1001F00003070F1E1C18100000060912141209062E
:1002000000060917170906001F111F001F111F0004
:100210001F111F001F1F1F001F1F1F001F111F0086
:100220001F1F1F001F1F1F00040E1F04041F0E04AA
:10023000010101050D1F0C0411040A11111F110009
:10024000110E111111110E000A00111111110E00E1
:100250000E11111611111610001C1F1F1F13101064
:10026000001C13111D13101000181711191710106E
:10027000001F11111F101010206D332020200000CE
:10028000204D4D4920200000204D4D02202000002F
:1002900020444343202000002053544F50200000AE
:1002A00053484F52542100002048414C5420000034
:1002B00020202020202000002050524F4720000006
:1002C0005245534554200000202054504D2000003A
:1002D000555044415445000020202020002533641F
:1002E00000252D31312E31317300252D3564002547
:1002F000632F256320256300256300462530326483
:100300003D25630020200102202020202020200005
:100310002533640025336400252D3564002D2D2DF3
:100320002D2020004144523A20256C6420202020BA
:1003300020202020202000232D007E0E0E0E0E1BDC
:100340001B1C0E1B1B7E0E0E0E0E636F72746F2035
:1003500028312E356D73292000006C756E676F2073
:1003600028342E3032356D7329004D6F746F726FE3
:100370006C61000000000000000044434320202086
:10038000202000000000000000004D4D2000000073
:100390000000000000000000000044434300000093
:1003A00000000000000000000000706F73697469B5
:1003B000766120284D4D290000006E6567617469E3
:1003C00076612028444343290000303A206F666656
:1003D00020202020202020202000313A2054616954
:1003E0006C626974732020202000323A202B20494F
:1003F000644E6F74696679202000333A202B2041C7
:1004000063636573736F72792000526970726973E8
:1004100074696E6120202020200053616C76612079
:100420002020202020202020200052697072697333
:1004300074696E6120202020200053616C76612059
:100440002020202020202020200020737461746F41
:10045000206C61796F757420200020737461746F53
:10046000206C61796F7574202000636F72746F2047
:1004700028312E356D73292020006C6172676F2042
:1004800028342E3032356D7329004D6F746F726FC2
:100490006C61000000000000000044434320202065
:1004A000202000000000000000004D4D2000000052
:1004B0000000000000000000000044434300000072
:1004C00000000000000000000000706F7369746994
:1004D000766120284D4D290000006E6567617469C2
:1004E00076612028444343290000303A2044657354
:1004F000616374697661646F2000313A20546169E8
:100500006C626974732020202000323A202B20492D
:10051000644E6F74696679202000333A202B2041A5
:1005200063636573736F72792000526573746175CC
:100530007261722020202020200047756172646162
:1005400072202020202020202000526573746175C5
:100550007261722020202020200047756172646142
:100560007220202020202020200020457374616408
:100570006F204D617175657461002045737461640D
:100580006F204D617175657461004B75727A20281A
:10059000312E356D7329202000004C616E672028B4
:1005A000342E3032356D732900004D6F746F726FC9
:1005B0006C61000000000000000044434320202044
:1005C000202000000000000000004D4D2000000031
:1005D0000000000000000000000044434300000051
:1005E00000000000000000000000706F7369746973
:1005F0007620284D4D29000000006E656761746902
:1006000076202844434329000000303A2061757366
:1006100020202020202020202000313A2054616911
:100620006C626974732020202000323A202B20490C
:10063000644E6F74696679202000333A202B204184
:1006400063636573736F72792000416E6C616765D7
:100650006E7A757374616E642000416E6C616765BB
:100660006E7A757374616E64200057696564657293
:100670006865727374656C6C6E005370656963684D
:1006800065726E2020202020200020776965646537
:100690007268657273742E20200020737065696320
:1006A0006865726E20202020200073686F727420AD
:1006B00028312E356D73292000006C6F6E6720285D
:1006C000342E3032356D732900004D6F746F726FA8
:1006D0006C61000000000000000044434320202023
:1006E000202000000000000000004D4D2000000010
:1006F0000000000000000000000044434300000030
:1007000000000000000000000000706F7369746951
:10071000766520284D4D290000006E65676174697B
:1007200076652028444343290000303A206F6666EE
:1007300020202020202020202000313A20546169F0
:100740006C626974732020202000323A202B2049EB
:10075000644E6F74696679202000333A202B204163
:1007600063636573736F72792000526573746F727F
:100770006520202020202020200053617665202045
:1007800020202020202020202000526573746F72CA
:100790006520202020202020200053617665202025
:1007A00020202020202020202000206C61796F75DF
:1007B00074207374617475732000206C61796F7597
:1007C000742073746174757320005B756E6B6E6F4B
:1007D000776E207374617475735D00466F726D611E
:1007E000746F20696E636F6D70617400466F726D17
:1007F00061746F20696E636F6D702E2000696E6B7F
:100800006F6D7061742E20466F726D617400696E39
:10081000636F6D7061742E20466F726D6174005B42
:10082000756E6B6E6F776E206572726F725D002EE3
:100830002E20617474656E64657265202E2E200012
:10084000233D63616E63656C6C6100000000000015
:10085000002876756F746F2900000000000000000A
:1008600000002E2E63616E63656C6C617A696F6E39
:10087000652E00206572726F726500000000000036
:100880000000000020736F6C6F2044434321202040
:100890002020202000207072696D61207072656DCB
:1008A0006920474F20002A3D416E6E756C6C6100D7
:1008B000000000000000002070726F6772616D6DB3
:1008C000617A696F6E6520002D636F72746F2063AB
:1008D0006972637569746F2D00206E617469766F3B
:1008E0002028313A312920202000206C696E656172
:1008F00072652028323A31292020002070726F67FB
:100900007265737369766F20312020002070726FDA
:10091000677265737369766F2032202000204D6FF7
:10092000646F204143202020202020202000204DE3
:100930006F646F20444320202020202020200020AE
:100940004175746F53746570202020202020200092
:100950002A6C656767692000000000000000000045
:10096000002A7363726976690000000000000000CD
:1009700000002E2E20736372697474757261202ECC
:100980002E20002E2E2E206C657474757261202E20
:100990002E2E2000212121206572726F7265202188
:1009A0002121202000204F4B20202020202020200B
:1009B0002020202020002E2073616C7661746167F6
:1009C00067696F202E20002E2E2072697072697365
:1009D00074696E6F202E2000233D43616E63202AD0
:1009E0003D416E6E756C202000233D5369202A3DE9
:1009F000416E6E756C6C6120200020636F6E6669BD
:100A0000677572617A696F6E6520005350454E5468
:100A10004F00000000000000000000002A204E658A
:100A20007373756E205472656E6F202A0020636F99
:100A300072746F20636972637569746F20002A2A6B
:100A40002A2074696D65206F7574202A2A2A004156
:100A500063636573732E20202534642F253464006E
:100A6000436F6E6669677572617A696F6E65202083
:100A70000020636F6E6669677572617A696F6E6573
:100A800020002E2E2E20657370657265202E2E2E6E
:100A9000202000233D626F7272617200000000002E
:100AA000000000002873696E2046696368612900B0
:100AB00000000000002E2E2E20626F7272616E64A4
:100AC0006F202E2E2E002046616C6C6F00000000FF
:100AD0000000000000000020736F6C6F20706172D6
:100AE00061204443432120002022474F222070727E
:100AF000696D65726F202020002A3D43616E636539
:100B00006C6172000000000000002050726F67727C
:100B1000616D6163696F6E202020002D636F7274B8
:100B20006F20636972637569746F2D00206E617444
:100B300069766F2028313A312920202000206C6905
:100B40006E6561722028323A312920202000207001
:100B5000726F677265737369766F20312020002091
:100B600070726F677265737369766F203220200030
:100B7000204D6F646F204143202020202020202022
:100B800000204D6F646F204443202020202020202F
:100B90002000204175746F53746570202020202040
:100BA0002020002A6C656572200000000000000013
:100BB000000000002A6573637269000000000000F5
:100BC00000000000002E2065736372696269656E23
:100BD000646F202E20002E2E2E206C6579656E64A9
:100BE0006F202E2E2E20002121212046616C6C6F5B
:100BF0002021212120202000204F4B2020202020B8
:100C00002020202020202020002E2E2067756172B9
:100C100064616E646F202E2E20002E207265737426
:100C2000617572616E646F202E2000233D426F72E9
:100C30007261202A3D43616E632E2000233D53697B
:100C4000202A3D43616E63656C6172200020436F12
:100C50006E66696775726163696F6E202000446516
:100C60007361637469766164612020202020002A0A
:100C70002A2A2053696E205472656E202A2A2A007F
:100C80002A636F72746F20636972637569746F2A67
:100C9000005469656D706F20657870697261646F6A
:100CA000200041636365732E202534642F2534644E
:100CB000000000436F6E66696775726163696F6EED
:100CC0002020200020436F6E66696775726163693A
:100CD0006F6E2020002E2E2E2077617274656E209C
:100CE0002E2E2E202000233D4CF6736368656E0087
:100CF00000000000000000286B65696E2045696EE9
:100D00007472616729000000202E2E2E206CF6736D
:100D1000636865202E2E2E2000204665686C657263
:100D200000000000000000000000206E75722066C8
:100D3000FC722044434321202020002065727374FC
:100D400020474F206472FC636B656E002A3D416250
:100D5000627275636800000000000000002050729D
:100D60006F6772616D6D696572756E6700002D2D1C
:100D7000204B75727A7363686C75DF202D2D00200F
:100D80004E617469762028313A31292020202000D4
:100D9000204C696E6561722028323A31292020206A
:100DA000002050726F67726573736976203120205E
:100DB00020002050726F677265737369762032204D
:100DC000202000204143204D6F6475732020202097
:100DD00020202000204443204D6F64757320202084
:100DE0002020202000204175746F537465702020EE
:100DF0002020202020002A6C6573656E0000000012
:100E0000000000000000002A736368722E000000DA
:100E100000000000000000002E2E20736368726541
:100E20006962656E202E2E00002E2E2E206C6573BA
:100E3000656E202E2E2E20200000212121204665C7
:100E4000686C657220212121200000204F4B20205A
:100E50002020202020202020202000002E2E207363
:100E6000706569636865726E202E2E000077696573
:100E70006465726865727374656C6C656E00233DA1
:100E80004CF6736368656E202A3D416262720023EE
:100E90003D4A61202A3D416262727563680000002C
:100EA000206CF6736368656E2020202020202020AF
:100EB0000041555300000000000000000000000049
:100EC00000002A2A206B65696E65204C6F6B202A12
:100ED0002A20002A2A204B75727A7363686C75DFAA
:100EE000202A2A002A205A656974FC62657273639D
:100EF00068722E2A00576569636865202534642F5F
:100F00002534640000004B6F6E666967757261740A
:100F1000696F6E20202000204B6F6E6669677572C6
:100F20006174696F6E2020002E2E2E207761697407
:100F3000696E67202E2E2E2000233D64656C65743B
:100F400065000000000000000000286E6F20656E44
:100F500074727929000000000000002E2E2E2064FB
:100F6000656C6574696E67202E2E2E002066617593
:100F70006C740000000000000000000000204443EA
:100F800043206F6E6C7921202020202020002070CB
:100F90007265737320474F20666972737400002A6C
:100FA0003D43616E63656C000000000000000000BE
:100FB0002070726F6772616D696E670000000000DB
:100FC000002D73686F727420636972637569742D84
:100FD0002000206E61746976652028313A3129201D
:100FE000202000206C696E6561722028323A312918
:100FF000202020002070726F6772657373697665B8
:1010000020312020002070726F67726573736976DB
:10101000652032202000204143204D6F6465202050
:1010200020202020202000204443204D6F64652094
:101030002020202020202000204175746F537465EB
:101040007020202020202020002A7265616420006A
:10105000000000000000000000002A77726974653B
:1010600000000000000000000000002E2E2E20775F
:10107000726974696E67202E2E2E20002E2E2E206F
:1010800072656164696E67202E2E2E200021212159
:10109000206661756C742021212120202000204FC2
:1010A0004B20202020202020202020202020002E27
:1010B0002E2E20736176696E67202E2E2E20200042
:1010C0002E2E20726573746F72696E67202E2E202B
:1010D00000233D44656C2E202A3D43616E63656CA0
:1010E0002000233D596573202A3D43616E63656C82
:1010F00020200020636F6E66696775726174696F86
:101100006E2020004F464600000000000000000056
:1011100000000000002A2A2A206E6F2054726169A4
:101120006E202A2A2A002A2073686F72742063694D
:10113000726375697420002A2A2A2074696D6520FB
:101140006F7574202A2A2A00506F696E742020253A
:1011500034642F253464000000436F6E6669677540
:10116000726174696F6E2020200020636F6E666963
:101170006775726174696F6E2020005B6E6F206D01
:101180006573736167655D004003A001CF00670070
:101190004400330019001000204D3320656E616259
:1011A0006C65642020202020003D253564003078C7
:1011B0002530386C580020253564002534646D7363
:1011C000002533642C25647300202E2E2E2E202023
:1011D00020202020202020002564206D7300202561
:1011E00032640025346400202D2D2D002020202085
:1011F00020202000204F4B20202020002533640099
:101200002D2D2D002534643A200025366400202D34
:101210002D2D2D2D0025346400202D2D2D0043561D
:101220003A253464204269743A25643D0043563AB5
:1012300020202020204269743A203D200025357569
:1012400000202D2D2D2D004142434445464748495D
:101250004A4B4C4D4E4F5051525354555657585976
:101260005A303132333435363738392E2C3A2D2B2B
:10127000232F3D3C7C3E20004D4D20492020313421
:1012800020004D4D20492020323761004D4D20492E
:101290002020323762004D4D2002202031342000C2
:1012A0004D4D20022020323761004D4D200220207C
:1012B000323762004443432020203134200044432D
:1012C000432020203238200044434320203132384C
:1012D00020006D3320202031323820003A200025B4
:1012E0003575005365724E722E2025386C750032AC
:1012F0002E302E3100536F6674772E205600253322
:1013000064004E723A202532642020004D656E75CF
:10131000204C6F636F6D6F746976650050726F67F4
:1013200072616D6D617A2E204443430050726F6785
:1013300072616D6D617A2E206D330000537461749B
:101340006F204C61796F757400000000496D706FFB
:1013500073746174696F6E65000000004C43442033
:10136000726574726F696C6C2E0000004C6F6B4379
:101370006F6E74726F6C000000000000557363693B
:1013800074610000000000000000000053656C65FF
:101390007A696F6E6120000000000000466F726D78
:1013A00061746F2044617469200000004E6F6D65A8
:1013B00020202020202000000000000056616C6FDB
:1013C00072652020202020000000000043562028C5
:1013D000627974652900000000000000435620284F
:1013E000626974290000000000000000496E642E4C
:1013F000205072696D6172696F000000496E642E41
:101400002045737465736F000000000052656769C2
:101410007374726F00000000000000005061676587
:101420002D4D6F6465000000000000004D61696E85
:1014300020547261636B0000000000005261696C0F
:10144000436F6D2043560000000000004D6F646F35
:101450002031323846530000000000004D6F646FA9
:10146000204A6F676469616C00000000496D706F0D
:101470007374617A2E2073383800000043616E6304
:10148000656C6C610000000000000000426F6F732B
:1014900074657200000000000000000056656C6F6B
:1014A0006369746120696E74657266004465632EB9
:1014B0004163636573736F7269000000466F726DFC
:1014C00061746F204C6F636F000000005061757392
:1014D00061207365676E2E4D4D200000537570704E
:1014E0006F72742E5261696C436F6D006D6F64751D
:1014F0006C69207338380000000000007465737454
:10150000206D6F64756C692073383800506F6C2ED5
:1015100020636F72746F636972632E0053656E731C
:101520002E20636F72746F6369722E005475747429
:1015300069206163636573736F726900466F726DD2
:101540002E206163636573736F7269006D696E2E1F
:10155000746D702E696D70756C736F006D61782E8F
:10156000746D702E696D70756C736F00696E64694F
:1015700072697A7A6F206D33000000004D656E75D8
:10158000204C6F636F6D6F746F72610050726F6784
:1015900072616D6D617220444343000050726F6749
:1015A00072616D6D6172206D33000000457374616E
:1015B000646F204D6171756574610000416A7573D7
:1015C000746573000000000000000000496C756D38
:1015D000696E6163696F6E204C4344004C6F6B43CE
:1015E0006F6E74726F6C00000000000053616C69D4
:1015F00072000000000000000000000053656C65F0
:101600006363696F6E61722000000000466F726D47
:1016100061746F204461746F730000004E6F6D62DF
:1016200072652020202000000000000046696368E9
:1016300061202020202000000000000043562028C8
:1016400062797465290000000000000043562028DC
:10165000626974290000000000000000446972659E
:101660006363696F6E20636F7274610044697265B1
:101670006363696F6E206C617267610052656769B0
:101680007374726F00000000000000005061676515
:101690002D4D6F646500000000000000456E20566F
:1016A0006961207072696E6369702E005261696CA5
:1016B000436F6D2043560000000000004D6F646FC3
:1016C00020313238207061736F7300004D6F646F8A
:1016D000206465206D616E646F000000416A75735F
:1016E000746573207338380000000000426F727216
:1016F000617200000000000000000000426F6F7384
:101700007465723A000000000000000041636365E8
:10171000736F72696F733A0000000000466F726D5C
:1017200061746F206465205472656E00506175733A
:1017300061205365F1616C204D4D00005375706F51
:10174000727465205261696C436F6D004D6F6475F2
:101750006C6F73207338380000000000507275659C
:101760006261204D6F642E2073383800506F6C2EEC
:1017700020436F72746F636972632E0053656E73DA
:101780002E20436F72746F6369726300546F646FCD
:10179000732041636365736F722E0000466F726D34
:1017A00061746F2061636365736F72004475726169
:1017B000632E496D70756C2E6D696E004475726193
:1017C000632E496D70756C2E6D6178004469726589
:1017D0006363696F6E206D33000000004C6F6B20F7
:1017E0004D656EFC00000000000000004443432DE6
:1017F00050726F6772616D6D672E00006D332050FF
:10180000726F6772616D6D672E000000416E6C61D2
:1018100067656E7A757374616E64000045696E73F6
:1018200074656C6C756E67656E0000004C434420F7
:1018300042656C6575636874756E67004C6F6B43C9
:101840006F6E74726F6C0000000000004578697460
:1018500000000000000000000000000041757377E8
:10186000E4686C656E20000000000000446174654F
:101870006E666F726D617400000000004E616D65F0
:1018800020202020202000000000000045696E7408
:1018900072616720202000000000000043562028CD
:1018A000627974652900000000000000435620287A
:1018B0006269742900000000000000004261736941
:1018C000732D416472657373650000006C616E670F
:1018D0006520416472657373650000005265676935
:1018E00073746572000000000000000050616765BD
:1018F0002D4D6F64650000000000000048617570A8
:1019000074676C6569730000000000005261696CC7
:10191000436F6D204356000000000000313238460E
:1019200053204D6F64650000000000005265676C35
:1019300065726D6F64757300000000007338382D98
:1019400045696E7374656C6C756E67004B6F6E667F
:10195000696775726174696F6E000000426F6F7322
:1019600074657200000000000000000057656963A4
:1019700068656E0000000000000000004C6F6B66A0
:101980006F726D6174000000000000004D4D2D531A
:1019900069676E616C205061757365005261696C96
:1019A000436F6D20537570706F7274007338382DEB
:1019B0004D6F64756C650000000000007338382DB1
:1019C0004D6F64756C746573740000004B75727AAA
:1019D0007363686C2E2D506F6C2E00004B75727AFD
:1019E0007363686C2E2D456D70662E00616C6C659E
:1019F000205765696368656E00000000576569637C
:101A000068656E666F726D61740000006D696E2EA0
:101A100020536368616C747A656974006D61782E17
:101A200020536368616C747A656974006D3320417A
:101A30006472657373650000000000004C6F636F93
:101A40006D6F74697665206D656E75004443432043
:101A500070726F6772616D6D696E67006D332070B3
:101A6000726F6772616D6D696E6700004C61796FAE
:101A70007574207374617475730000005365747419
:101A8000696E677300000000000000004C434420B2
:101A90006261636B6C696768740000004C6F6B4334
:101AA0006F6E74726F6C00000000000045786974FE
:101AB00000000000000000000000000053656C659D
:101AC00063742000000000000000000044617461A5
:101AD00020666F726D617400000000004E616D65DC
:101AE000202020202020000000000000456E74729D
:101AF00079202020202000000000000043562028EC
:101B00006279746529000000000000004356202817
:101B10006269742900000000000000005072696DC5
:101B200061727920616464726573730045787465CD
:101B30006E642E2061646472657373005265676918
:101B4000737465720000000000000000506167655A
:101B50002D4D6F6465000000000000004D61696E4E
:101B600020747261636B0000000000005261696CB8
:101B7000436F6D20435600000000000031323846AC
:101B800053204D6F64650000000000004A6F6764D9
:101B900069616C204D6F6465000000007338382067
:101BA00073657474696E67730000000044656C654A
:101BB000746500000000000000000000426F6F73B9
:101BC000746572000000000000000000506F696E34
:101BD0007473000000000000000000004C6F632ED2
:101BE00020666F726D617400000000004D4D20731F
:101BF00069676E616C207061757365005261696C14
:101C0000436F6D20537570706F7274007338382095
:101C10006D6F64756C6573000000000073383820C8
:101C20006D6F64756C6520746573740053686F72B2
:101C30007420632E20706F6C2E00000053686F724A
:101C40007420632E2073656E732E0000616C6C200F
:101C5000506F696E7473000000000000506F696E71
:101C6000747320666F726D61740000006D696E2E72
:101C70007377697463682E74696D65006D61782E81
:101C80007377697463682E74696D65006D332061C4
:101C9000646472657373000000000000202020302F
:101CA000782530386C582020200011241FBECFEF3B
:101CB000D0E1DEBFCDBF11E0A0E0B1E0E0EEFEE993
:101CC00000E00BBF02C007900D92A23DB107D9F70B
:101CD00014E0A2EDB1E001C01D92A238B107E1F716
:101CE0000E94940E0C946E4F0C9400008091D201CF
:101CF000089581E08093D301089580E00E94F71653
:101D0000BC018FEF6F3F780719F080E00E940A3026
:101D10000E94A3270E94CE198091D301882311F439
:101D20000E949315A8950895CF93DF930E946E2685
:101D30000E94700F83E068E04EE422E00E94E62DEE
:101D40000E943E1178940E946B130E944125DC0191
:101D500014968C910E948E1582E067EF70E00E94CD
:101D6000D9170E945925823021F00E9459258130CF
:101D700021F482E063EF70E007C00E9459258038AB
:101D8000D9F482E06FEE70E00E94D91781E060E044
:101D90000E94111682E066E50E94061782E062ED5D
:101DA00070E00E94D9170E944125EC0181E00E9459
:101DB0004114882349F125C00E94592500D000D044
:101DC0000F92EDB7FEB7319692E0ADB7BEB7119660
:101DD0009C9328EE30E032832183838314820E9417
:101DE0007F170F900F900F900F900F9081E060E0A1
:101DF0000E94111682E068ED70E00E94D917A89544
:101E0000FECF80E00E94552682E00E944114882384
:101E100019F084E00E94552683E00E944114882333
:101E200019F085E00E94552684E00E944114882321
:101E300029F081E00E94552601C0A8950E94F02754
:101E40008823D9F389859A85009749F060E070E08E
:101E500040E050E00E944F2DBC01009711F46A81D0
:101E60007B818FEF0E94012681E011C00E944B20F0
:101E70000E946514BFEF8F3F9B07C1F70E947D0E44
:101E80008091D3018823A1F31092D30180E00E94B6
:101E9000541BEECF9091D201981701F19630F1F0DA
:101EA000953011F48630D1F48093D201853029F435
:101EB00080E060E245E00E9420278091D2018630D8
:101EC00029F480E060E246E00E9420278091D20160
:101ED0000E94CD2F81E08093D301089580E0089582
:101EE0008FE78ABB1BBA80E187BB18BA80EF84BB3F
:101EF0008FEF85BB8BEB81BB8CEC82BB82E082B920
:101F000087EF83B987E78093610081EE8093620059
:101F100087E18093640089E1809365000E9420122C
:101F2000A89588E181BD8EE081BD0895DC01909186
:101F3000D70189E0989FF0011124EF52FC4F90E007
:101F40008D9181939F5F9930D9F78091D7018F5FF1
:101F50008093D7018091D701843010F01092D7017F
:101F600008951F920F920FB60F920BB60F92112485
:101F70001F932F933F934F935F936F937F938F9311
:101F80009F93AF93BF93EF93FF9380910001909144
:101F900001012FEF8F3F920761F0BB9A8FB9769BBB
:101FA0000BC0BB981092D6011092DC011092DB019D
:101FB00003C0BB988FEF8FB91FB117FF8AC0809104
:101FC000DD019091DE01892BE1F08091D9018F5FD5
:101FD0008093D9018091D901803210F01092D901FB
:101FE0009091D9018091DA01981759F48091DA0122
:101FF0008F5F8093DA018091DA01803210F01092C5
:10200000DA018091DB019091DC01815D934061F008
:1020100058F08091D8018F5F8093D8018091D801CA
:10202000843010F01092D8011092DE011092DD0180
:102030001092DC011092DB0180910201181721F44B
:1020400081E08093D60177C01092D601412F50E0F5
:102050004F775070682F70E04617570729F01F3FE1
:1020600019F08F3F09F067C08091D90129E0829F64
:10207000C00111248F549D4F9093DE018093DD01A8
:102080004617570709F057C09091D7018091D801A2
:10209000981721F488EA92E00E94960F8091D80167
:1020A00029E0829FC00111248F529C4F9093DC0144
:1020B0008093DB018091D8018F5F8093D80180915C
:1020C000D801843010F01092D80189E08093D401B7
:1020D00032C02091D601213029F0213060F1263024
:1020E00050F515C082E08093D601103419F4109297
:1020F000D50121C0113419F42093D5011CC012342C
:1021000019F0133491F483E08093D50114C0E22FC9
:10211000F0E08091D50190E002968E179F0744F081
:10212000E352FE4F8081181719F01092D60103C0B8
:102130002F5F2093D6018091D601882329F0109338
:1021400000011092010121C0E091DB01F091DC015E
:102150003097A9F081918093000110920101F093D2
:10216000DC01E093DB018091D40181508093D401A4
:10217000882359F41092DC011092DB0106C08FEF26
:102180009FEF9093010180930001E091DD01F091B8
:10219000DE01309749F083E0E13DF80728F4119320
:1021A000F093DE01E093DD01FF91EF91BF91AF91DC
:1021B0009F918F917F916F915F914F913F912F915F
:1021C0001F910F900BBE0F900FBE0F901F90189590
:1021D0001F93AC011FB7F8942091D7018091D801CB
:1021E00030E090E001972817390741F08091D7013E
:1021F000833039F48091D801882319F41FBF80E01F
:1022000005C0CA010E94960F1FBF81E01F9108956B
:10221000DC01E8EAF2E08D91819382E0E13BF8078E
:10222000D1F708959C01009739F14FB7F894909138
:10223000D9018091DA01981721F44FBF20E030E0F6
:102240001BC09091DA0189E0989FF0011124EF54AE
:10225000FD4FD90190E081918D939F5F9930D9F71F
:102260008091DA018F5F8093DA018091DA01803208
:1022700010F01092DA014FBFC90108950E944B255A
:10228000262F2F772093E20147E096958795779543
:1022900067954A95D1F7262F2F772093E10137E0F4
:1022A00096958795779567953A95D1F7262F2F774D
:1022B0002093E00127E096958795779567952A9575
:1022C000D1F76F776093DF0187B3807F87BB88B3D7
:1022D000807F88BB84EE8DB90895882351F080916A
:1022E000650084608093650000000000000000002D
:1022F0000895809165008B7F8093650008950F930A
:102300001F93DF93CF930F92CDB7DEB7182F8AB309
:10231000807F8ABB80E00E946D11809165008260A1
:1023200080936500112321F080916500816003C0D6
:10233000809165008E7F809365000000000081E041
:102340000E946D1109B380E00E946D1110E084E0DD
:10235000000F111F8A95E1F7000000000000000047
:1023600081E00E946D1199B39F70902B80E099835A
:102370000E946D118AB38F608ABB9981892F0F905B
:10238000CF91DF911F910F91089580E00E947F11FE
:10239000982F87FF11C08091E6019091E70128E016
:1023A0008130920714F080E0089501969093E70140
:1023B0008093E60181E008958091E801882319F473
:1023C0009F779093E9011092E7011092E60180E077
:1023D00008959B01AC018091F7039091F803A091BF
:1023E000F903B091FA0382179307A407B50798F091
:1023F0008091F7039091F803A091F903B091FA034B
:1024000060E0821B930BA40BB50B80509041A04061
:10241000B040A0F412C08091F7039091F803A0910E
:10242000F903B091FA0360E0281B390B4A0B5B0BF0
:102430002050304F4F4F5F4F08F061E0862F0895D6
:1024400010927D0080B7877F80BF17BE11BE89E6DE
:1024500083BF8BE085BD8FE183BD87B7806887BF71
:102460000895EF92FF920F931F932091F7033091FD
:10247000F8034091F9035091FA037C0100E010E069
:10248000E20EF31E041F151F01C0A895C801B70175
:102490000E94E9118823C9F31F910F91FF90EF90DB
:1024A0000895FF920F931F93082F162FF42E8091FB
:1024B00065008D7F8093650080E00E946D118AB376
:1024C0008F608ABB8BB3902F92959F70807F982BE3
:1024D0009BBB112321F080916500816003C0809136
:1024E00065008E7F8093650081E00E946D1180E021
:1024F0000E946D11FF2029F088E090E00E943112C7
:102500000FC08BB30F70807F802B8BBB000000004F
:102510000000000081E00E946D1180E00E946D11BA
:102520001F910F91FF900895EF92FF920F931F93C9
:102530002091F7033091F8034091F9035091FA0389
:102540007C0100E010E0E20EF31E041F151F02C024
:102550000E947D0EC801B7010E94E9118823C1F3D2
:102560001F910F91FF90EF9008951F920F920FB659
:102570000F920BB60F9211241F932F933F934F93FB
:102580005F936F937F938F939F93AF93BF93EF93DB
:10259000FF938091E301882309F089C081E0809353
:1025A000E30178948091E5018F5F8093E50180914C
:1025B000E50190E083709070009719F0019741F564
:1025C00016C08091F7039091F803A091F903B091A0
:1025D000FA030196A11DB11D8093F7039093F803B0
:1025E000A093F903B093FA030E944D1411C0809197
:1025F000F7039091F803A091F903B091FA03817069
:102600009070892B19F00E947F1402C00E9405145B
:102610008091E401882321F00E94C5118093E40198
:102620008091E401882309F040C09091FB038091E0
:10263000FC039817B9F18091FC03E82FF0E0E55016
:10264000FC4F9281182F1F5F103108F010E0903876
:1026500001F58091FB03811729F1E12FF0E0E550AE
:10266000FC4F92819F3F19F49091E901906897FF88
:1026700002C01092E801892F807C803419F481E037
:102680008093E8011F5F103108F010E0892F60E0AF
:1026900002C0892F61E040E00E9451121093FC03B8
:1026A00081E001C080E08093E4011092E301FF919A
:1026B000EF91BF91AF919F918F917F916F915F91BA
:1026C0004F913F912F911F910F900BBE0F900FBE16
:1026D0000F901F901895CF93DF9388E290E00E94AF
:1026E000311280E360E041E00E94511280E360E03B
:1026F00041E00E94511280E360E041E00E945112EB
:1027000080E260E041E00E94511288E20E94FB15E5
:1027100080E40E94FB158AE00E94CE1589E20E94A7
:10272000FB158CE10E94FB1582E50E94FB1589E6F2
:102730000E94FB1584E70E94FB1580E40E94FB15B4
:1027400085E10E94CE1588E20E94FB1580E40E947C
:10275000FB150E940218EC0101C0A8959091FB03A3
:102760008091FC039817C9F70E94C5118823A9F727
:1027700081E00E947F118A3019F481E089AB01C0A9
:1027800019AA88E00E94FB1581E00E94FB1586E0F3
:102790000E94FB158CE00E94FB1580E060E00E9427
:1027A000111680E06CE171E00E94F21681E060E6B3
:1027B00071E00E94F21682E068E671E00E94F21673
:1027C00083E068E771E00E94F216DF91CF910895EF
:1027D0009091EC01E92FF0E0E451FE4F82839F5F7E
:1027E0009093EC01983010F01092EC019091ED0173
:1027F0008091EC01981741F4892F8F5F8093ED0150
:10280000883010F01092ED01089531B12091EB0164
:10281000220F36FD2160822F83708150823028F490
:1028200024FF02C02E6001C0217F2093EB01909114
:10283000EA01990F37FD9160892F837081508230B2
:1028400028F494FF02C09E6001C0917F9093EA013A
:10285000207C892F807C203831F4882341F0803C13
:1028600079F48AE105C0203459F4803C21F489E1EF
:102870000E94E8130895882319F48AE10E94E8135E
:102880000895893110F080E00895E82FF0E0EA50D3
:10289000FE4F8081811181E008953091280234300B
:1028A00029F485B3806F85BB97980895979A25B3CF
:1028B00080E190E002C0880F991F3A95E2F7809579
:1028C000807F2F70822B85BB08959091ED018091C0
:1028D000EC01891719F42FEF3FEF0FC0E92FF0E05B
:1028E000E451FE4F8281282F30E0892F8F5F809343
:1028F000ED01883010F01092ED01C90108958F921A
:102900009F92AF92BF92CF92DF92EF92FF920F937E
:102910001F93CF93DF930E94760E982F8091290208
:10292000981729F09093290282E20E94E81383B35A
:10293000E1B0EE0CEE0C90E1E9228F70E82ACC2495
:10294000DD2495E0892E81E0A82EB12C9924939462
:10295000E0912802E89DF0011124EC0DFD1DED5FD2
:10296000FE4FF49088E18F1508F481C00E2D0A25E2
:102970000170CF2DD0E0FE01E15FFD4F1081110FFE
:102980000E945925803819F4002371F009C0011103
:102990001160812F90E0817190708131910511F467
:1029A0001F6103C0892B09F4107E812F90E080768F
:1029B00090708034910519F41F7182E00CC0803250
:1029C000910519F4106E81E006C08036910511F072
:1029D00080E001C083E0FE01E15FFD4F10838230A3
:1029E00099F0833059F1813009F041C096E1F91630
:1029F00021F480910B02882319F48F2D0E94E81393
:102A0000CA50DE4F988233C0CA50DE4F18828F2DD5
:102A100080680E94E8130E94760E853041F585E1BA
:102A2000F81619F480910C0205C096E1F916F9F434
:102A300080910B028823D9F486E017C0FE01EA508A
:102A4000FE4F80818F5F8083882309F490828BEE14
:102A5000F80E91E09F1558F080910B02893738F0FD
:102A600080910C02893718F085E00E944A0F089483
:102A7000C11CD11C85E0C816D10411F0E69468CFC2
:102A8000809128028F5F80932802853010F0109289
:102A90002802DF91CF911F910F91FF90EF90DF906F
:102AA000CF90BF90AF909F908F90089590932804FF
:102AB00080932704892B89F1709326046093250461
:102AC0008091F7039091F803A091F903B091FA0374
:102AD0009B0140E050E0280F391F4A1F5B1F2093E5
:102AE00021043093220440932304509324048091C2
:102AF00020048E7F80932004211531054105510566
:102B000061F481E090E0A0E0B0E080932104909334
:102B10002204A0932304B09324040895813308F081
:102B200080E381BF08958091270490912804892B28
:102B3000A1F160912104709122048091230490916D
:102B400024040E94E911882341F180912004E0913E
:102B50002704F0912804817009958091200491E068
:102B60008927809320042091F7033091F803409146
:102B7000F9035091FA038091250490912604A0E076
:102B8000B0E0820F931FA41FB51F80932104909380
:102B90002204A0932304B093240408951F93182FB4
:102BA00003C00E94A327A8952091FB038091FC03FA
:102BB00030E090E001972817390799F38091FB03E3
:102BC0008F3021F48091FC03882359F3F894E0912D
:102BD000FB03F0E0E550FC4F12838091FB038F5F15
:102BE0008093FB038091FB03803110F01092FB0374
:102BF00078941F9108951F93182F80E80E94CE1596
:102C0000812F0E94CE151F910895109228041092D2
:102C1000270481E00E94FB1508958CE00E94FB15BB
:102C200008958295880F880F807C860F80680E94A7
:102C3000FB150895BF92CF92DF92EF92FF920F9310
:102C40001F93CF93DF93C82EB62E8A0110922804CB
:102C50001092270421E02817A0F13FE0361788F1F1
:102C60004115510571F1FA0101900020E9F7319702
:102C7000DE2ED41A80E18D1510F490E1D92E8C2D22
:102C80006B2D0E941116E8018DE0E82E84E0F82EED
:102C900008C08881F70181937F01699182E00E94D9
:102CA00006179E01201B2D15A0F3C0921D04B092A3
:102CB0001E04D0921F0484E996E164EF71E00E9443
:102CC0005615DF91CF911F910F91FF90EF90DF90FC
:102CD000CF90BF900895DF93CF93CDB7DEB7A09785
:102CE0000FB6F894DEBF0FBECDBFDE0111969E0178
:102CF000205E3F4F04C09D93A217B30731F0FA0145
:102D00004F5F5F4F94919923B1F71C92AE014F5FD3
:102D10005F4F0E941A16A0960FB6F894DEBF0FBE42
:102D2000CDBFCF91DF9108950F931F93CF93DF9382
:102D3000082F80911D0460911E040E94111610E05E
:102D4000CDE0D4E009C0002311F460E201C0699134
:102D500082E00E9406171F5F80911F04181798F3E6
:102D6000DF91CF911F910F9108950E9411168EE06F
:102D70000E94FB150895EF92FF920F931F93CF933C
:102D8000DF93382F7B01122F883028F5483018F553
:102D9000842F90E0820F911D099714F018E0141B06
:102DA000330F330F330F340F832F80640E94FB15D2
:102DB000C0E0D0E0012F10E008C0F701EC0FFD1FCC
:102DC000E4918E2F0E94CE152196C017D107ACF347
:102DD0008FEF0E94FB15DF91CF911F910F91FF9014
:102DE000EF90089540E028E00E94BB1608958823E4
:102DF00041F0833019F02FEF3FEF06C00E946514B9
:102E000002C00E94582F9C01C90108951F93162FDC
:102E1000882309F45EC0823009F05EC067FF55C0A8
:102E20000E940218FC0181A98823E1F0143E11F4EC
:102E300014E84BC0163F11F414E947C01C3F11F4CD
:102E400011E843C0143C11F41EE83FC0163D11F4D4
:102E500019E93BC01C3D11F41AE937C0113F69F56F
:102E60001BE933C0143E11F411EE2FC0163F11F4CC
:102E70001FEE2BC01C3F11F415EF27C0113F11F4BA
:102E80001EEE23C0143C39F484E068E372E00E9433
:102E9000F21614E01AC0163D39F485E060E472E0E1
:102EA0000E94F21615E011C01C3D39F486E068E47A
:102EB00072E00E94F21616E008C01F3D31F487E070
:102EC00060E572E00E94F21617E0812F0E94CE1595
:102ED00003C0862F0E94282F1F9108951F93CF9320
:102EE000DF93182FEB0104C02196812F0E94061753
:102EF00068816623C9F7DF91CF911F9108950F93E1
:102F00001F93DF93CF93CDB7DEB7C055D0400FB638
:102F1000F894DEBF0FBECDBF9E01265A3F4F8E01F3
:102F20000F5F1F4FC8016A966EAD7FAD6A97A9010A
:102F30000E947A4C68968FAD6897B8010E946E1710
:102F4000C05BDF4F0FB6F894DEBF0FBECDBFCF9191
:102F5000DF911F910F9108950F931F93DF93CF93EC
:102F6000CDB7DEB7C055D0400FB6F894DEBF0FBE68
:102F7000CDBF9E01265A3F4F8E010F5F1F4FC801E4
:102F80006A966EAD7FAD6A97A9010E94514C689612
:102F90008FAD6897B8010E946E17C05BDF4F0FB608
:102FA000F894DEBF0FBECDBFCF91DF911F910F917F
:102FB00008951F93CF93DF93182FEB0104C0812F47
:102FC0000E9406172196FE0164916623C1F7DF91E6
:102FD000CF911F910895E82FF0E0EF70F070E65C5C
:102FE000FC4FE4918E2F90E0089590E083709070F4
:102FF000009731F0039711F48CE1089584E008956F
:103000008FE008958FE292E0089580914B0282FF55
:1030100005C08091310290913202089580912F0273
:1030200090913002089590914B0291FD19C092FF4A
:1030300005C080912904823099F404C0809129044C
:103040008F3071F4109229049260977F90934B0215
:1030500010924F0280E090E060E070E00E94561510
:1030600008958823E9F082E068EA71E00E94F21690
:1030700083E060EB71E00E94F21684E068EB71E09F
:103080000E94F21685E060EC71E00E94F21686E084
:1030900068EC71E00E94F21687E060ED71E01CC000
:1030A00082E068E671E00E94F21683E068E771E072
:1030B0000E94F21684E068E871E00E94F21685E052
:1030C00060E971E00E94F21686E068E971E00E9412
:1030D000F21687E060EA71E00E94F216089580918E
:1030E0002E02833014F010922E0280912E028F5FF8
:1030F00080932E028150813041F0823061F088232C
:1031000079F481E060E772E003C081E068E672E094
:103110000E94F216089581E060E672E00E94F216C5
:103120000895882321F082E060EF71E003C082E01F
:1031300068EE71E00E94F2160895882321F081E084
:1031400060EE71E003C081E068ED71E00E94F2166C
:103150000895FF920F931F93DF93CF9300D000D079
:1031600000D0CDB7DEB78C01F62EFE01319686E099
:10317000DF011D928A95E9F7D8016D917C91CF010D
:103180000E94AA26F801808D918DA28DB38D282FE3
:103190002F772B8337E0B595A795979587953A9527
:1031A000D1F7282F2F772C8327E0B595A7959795F2
:1031B00087952A95D1F781708D83FF2011F0806863
:1031C0008D8380E06BE1AE014F5F5F4F0E940A2765
:1031D00026960FB6F894DEBF0FBECDBFCF91DF911C
:1031E0001F910F91FF90089580935F020E94790EC6
:1031F000089520914B0221FD0EC02B7F216020936A
:103200004B02909332028093310270933A026093A2
:1032100039020E94790E0895E0912F02F091300258
:103220008E179F0711F0EF2BF1F49B0140E050E067
:10323000A901332722278091350290913602A0916F
:103240003702B0913802A070B070282B392B4A2B6E
:103250005B2B209335023093360240933702509314
:1032600038020E94790E0895FC0180912F029091FE
:103270003002E817F90711F510924E0260934D02E3
:1032800060E070E08091350290913602A0913702A3
:10329000B091380280709070482B592B6A2B7B2B91
:1032A000222311F0616001C06E7F4093350250937C
:1032B000360260933702709338020FC0809131025A
:1032C00090913202E817F90751F410924E02609380
:1032D0004D0250933A02409339020E94790E0895AC
:1032E0001F93182F80E06CE00E941116112309F142
:1032F00000D000D00F92EDB7FEB7319682E0ADB7A7
:10330000BEB711968C938DED92E09283818380916C
:103310004F0290E08F779070948383830E947F1791
:103320000F900F900F900F900F9080E00E94CE159D
:1033300005C082E068ED72E00E94D9171F910895E0
:10334000EF92FF920F931F93182F80FF02C083E02C
:1033500001C085EA0E94CE15E12E11FF02C084E073
:1033600001C085EA0E94CE15E2FE02C085E001C0E0
:1033700085EA0E94CE15E3FE02C086E001C085EA20
:103380000E94CE15E4FE02C087E001C085EA0E94DB
:10339000CE151F910F91FF90EF90089560913B0221
:1033A00070913C0280913D0290913E026115710541
:1033B0008105910561F00E94E911882341F0109286
:1033C0003B0210923C0210923D0210923E0260912C
:1033D0003F0270914002809141029091420261153A
:1033E00071058105910571F00E94E911882351F062
:1033F00010923F021092400210924102109242023B
:103400000E94790E609143027091440280914502BE
:1034100090914602611571058105910561F00E9448
:10342000E911882341F01092430210924402109255
:1034300045021092460280914E0218166CF42091BB
:103440004D0230E02F7730708091500290E02817C5
:10345000390714F010924E0280914E0287FF09C086
:1034600080914D0290E08F779070892B11F410922B
:103470004E0280914E0220912A0230912B024091FF
:103480002C0250912D02882381F42115310541052C
:10349000510511F00E94790E10922A0210922B020F
:1034A00010922C0210922D0208952115310541052C
:1034B000510539F0CA01B9010E94E911882309F4C4
:1034C0006CC080914E02181644F40E94760E833030
:1034D00049F480914D028F5F03C080914D0281506D
:1034E00080934D0280914E02813059F08F3F49F018
:1034F000823061F08E3F51F028E833E140E050E047
:1035000009C020E335E740E050E004C020EE3EE291
:1035100040E050E0809150028E3781F48091F703B3
:103520009091F803A091F903B091FA03F7E0569552
:10353000479537952795FA95D1F721C08E3081F4BC
:103540008091F7039091F803A091F903B091FA03E9
:10355000E4E05695479537952795EA95D1F70FC042
:103560008091F7039091F803A091F903B091FA03C9
:1035700075E056954795379527957A95D1F7280F99
:10358000391F4A1F5B1F20932A0230932B0240935E
:103590002C0250932D020E94790E089580914B02C7
:1035A00080FD25C060913B0270913C0280913D02FC
:1035B00090913E02611571058105910521F00E94EF
:1035C000E9118823A1F01092320210923102109278
:1035D0005202109251021092300210922F02109259
:1035E0004B02109253020E94790E81E0089580E010
:1035F00008951F93FC01009769F410924B021092FA
:103600003B0210923C0210923D0210923E020E9438
:10361000CE1A48C070914B0271FD44C060934D02B8
:10362000CA01A0E0B0E0209135023091360240910D
:1036300037025091380220703070822B932BA42BCC
:10364000B52B8093350290933602A0933702B09346
:1036500038028091F7039091F803A091F903B0919B
:10366000FA0388519C4FAF4FBF4F816080933B025C
:1036700090933C02A0933D02B0933E0272FF09C0BA
:1036800071607B7F70934B02F0933202E0933102C2
:1036900007C07E7F70934B02F0933002E0932F02BD
:1036A0000E94790E1F910895DF92EF92FF920F937F
:1036B0001F9310915F02112399F081E060E00E9456
:1036C0001116812F81500E94F424BC0182E00E94D7
:1036D000D91710925F0288EE93E00E94941202C004
:1036E000882319F00E94051604C080E060E00E9463
:1036F000111680912F0290913002892BF9F00E94CF
:103700004125FC0140912F0250913002828193812A
:103710008417950749F42185328580915102909153
:1037200052022817390751F0538342838091510286
:1037300090915202928781870E942C2620912F021D
:103740003091300221153105C9F4109235021092E2
:103750003602109237021092380210924E021092E6
:103760003A021092390210924D0210924F0280914B
:103770004B028F7E80934B0210924C0280914B0241
:1037800082FD0DC08091470290914802A0914902AC
:10379000B0914A020097A105B10531F430C082E032
:1037A00067E373E00E94D9178DB79EB707970FB6EE
:1037B000F8949EBF0FBE8DBFEDB7FEB7319682E085
:1037C000ADB7BEB711968C9384E293E09283818368
:1037D0008091470290914802A0914902B0914A021B
:1037E00083839483A583B6830E947F17EDB7FEB7CA
:1037F00037960FB6F894FEBF0FBEEDBF51C021152E
:10380000310531F482E06DE173E00E94D91721C0E7
:1038100000D000D00F92EDB7FEB7319682E0ADB781
:10382000BEB711968C9388E193E0928381833483B1
:1038300023830E947F1780914B020F900F900F906F
:103840000F900F9080FF02C081E001C080E20E94D3
:10385000CE1510914C020E94760E682F863008F02B
:103860006150633091F480912F0290913002892B46
:1038700061F0612F70E06370707003E0660F771F76
:103880000A95E1F768587D4F08C070E013E0660FB5
:10389000771F1A95E1F768567D4F82E00E94D9178D
:1038A00080E06CE00E94111680914B0283FF12C0F1
:1038B00000D000D00F92EDB7FEB7319682E0ADB7E1
:1038C000BEB711968C9384E193E0928381838091BB
:1038D0004F0211C000D000D00F92EDB7FEB7319665
:1038E00082E0ADB7BEB711968C9380E193E09283EE
:1038F000818380914D0290E08F77907094838383D1
:103900000E947F170F900F900F900F900F90809153
:103910002F0290913002892B89F080914C028370A4
:10392000813081F487E10E944114882339F080E0DE
:103930000E94CE1580E068E272E05BC080E20E94E7
:10394000CE1559C080E00E94CE150E944125FC0191
:10395000808185FF43C080914D0287FF04C080E0D5
:103960006CE271E003C080E060E371E040E024E0DD
:103970000E94BB1680914E028823E1F018163CF09D
:103980008E3F81F08F3F94F48D3FA9F507C08230C0
:10399000C9F082309CF0833071F518C080E06CE48F
:1039A00071E017C080E068E471E013C080E064E477
:1039B00071E00FC080E064E371E00BC080E068E379
:1039C00071E007C080E06CE371E003C080E060E478
:1039D00071E044E024E00E94BB160DC080914D02CE
:1039E00087FF04C080E06CE171E003C080E064E226
:1039F00071E00E94F2160E94760E813049F489E04F
:103A00000E941125AC0181E060E00E946B1603C2A8
:103A100080914B0283FD06C080E060E040E050E012
:103A20000E941A1680914B0287FD03C000E010E04F
:103A300014C08091310290913202892B19F001E07B
:103A400010E00BC080914C020E94F51720E030E09E
:103A5000853010F021E030E08901F02E81E060E057
:103A60000E9411168091470290914802A09149024C
:103A7000B0914A020097A105B10509F429C18DE072
:103A80000E944114882329F48EE00E944114882367
:103A900081F100D00F9282E0EDB7FEB7818384E020
:103AA00093E0938382830E947F170F900F900F9073
:103AB0008DE00E944114882369F081E060EE71E09E
:103AC0000E94F21682E068EE71E00E94F2168DE923
:103AD00098E10CC081E068ED71E00E94F21682E08E
:103AE00060EF71E00E94F21681E998E16CE271E00A
:103AF000ECC087E00E941125BC0182E00E94D9172A
:103B000087E00E9411250E94314C182F04C080E2EA
:103B10000E94CE151F5F1031D0F310914C02812FFF
:103B20000E94F51790E0A0E0B0E0209147023091AC
:103B300048024091490250914A0282179307A40714
:103B4000B5070CF44DC081E06BE00E941116609146
:103B500047027091480281E090E0A0E0B0E0062EBC
:103B600004C0880F991FAA1FBB1F0A94D2F7209187
:103B7000350230913602409137025091380282234B
:103B80009323A423B5230097A105B10519F425EAD1
:103B900030E002C023E030E08DB79EB707970FB644
:103BA000F8949EBF0FBE8DBFEDB7FEB7319682E091
:103BB000ADB7BEB711968C938BEF92E09283818361
:103BC000CB0163839483368325830E947F17EDB7EF
:103BD000FEB737960FB6F894FEBF0FBEEDBFC0C05C
:103BE0001370133009F0BCC08FE00E944114882389
:103BF00051F480E10E944114882329F48CE00E9452
:103C00004114882369F180E10E944114882321F046
:103C100081E060E672E003C081E068E572E00E9446
:103C2000F21681E06FE00E94111600D000D00F92D2
:103C3000EDB7FEB7319682E0ADB7BEB711968C9363
:103C400088EF92E09283818381E090E09483838384
:103C50000E947F170F900F900F900F900F90DBC076
:103C600081E060E672E00E94F21681E06BE00E9463
:103C70001116EDB7FEB739970FB6F894FEBF0FBE19
:103C8000EDBF319682E0ADB7BEB711968C938FEE43
:103C900092E09283818386E090E09483838387E03F
:103CA00090E09683858381E090E0908787830E94EF
:103CB0007F17EDB7FEB739960FB6F894FEBF0FBE6B
:103CC000EDBF8FE698E168EC70E00E945615A3C046
:103CD00020913102309132022115310539F100D0A5
:103CE00000D00F92EDB7FEB7319682E0ADB7BEB708
:103CF00011968C938AEE92E092838183348323839E
:103D00000E947F170F900F900F900F900F9080914F
:103D100039028F710E94A019002321F08CE30E94C8
:103D2000CE152DC080E20E94CE151CC000D000D060
:103D30000F92EDB7FEB7319682E0ADB7BEB71196E0
:103D40008C9381EE92E09283818383E592E0948369
:103D500083830E947F170F900F900F900F900F900A
:103D6000FF2069F480913F0290914002A0914102AE
:103D7000B09142020097A105B10509F444C08091B9
:103D8000310290913202892BF1F580914C020E9410
:103D9000F5178530C0F181E060E00E94111686E4DD
:103DA0000E94CE15B2E0EB2EF12C012D112DDD2459
:103DB000D3948091350290913602A0913702B09150
:103DC00038028E219F21A023B1230097A105B105C0
:103DD00049F0B9E0BD1518F08D2D805D04C08D2D22
:103DE000885001C085EA0E94CE15D394E0E1DE162A
:103DF00029F0EE0CFF1C001F111FDBCF80E20E9498
:103E0000CE1581E006C0809135028F710E94A01905
:103E100080E00E9431181F910F91FF90EF90DF908A
:103E20000895CF93DF93EB0180934C02E82FF0E0ED
:103E3000EF70F070E65CFC4FE491E0935002611586
:103E4000710559F0CB0160E070E043E552E00E945B
:103E50004F2DD0935202C09351020E94790EDF91F0
:103E6000CF910895AC0180914B028C7F80934B02DF
:103E70001092520210925102662309F045C010922E
:103E8000530220912F02309130022115310521F08B
:103E9000309334022093330210923502109236028E
:103EA000109237021092380210923A0210923902A0
:103EB00010923202109231021092300210922F02B0
:103EC00010924E0210924C02109229044115510595
:103ED00051F18FEFBA010E94012680914B0281FDC2
:103EE00022C01092350210923602109237021092C0
:103EF0003802109232021092310210923002109267
:103F00002F0210924C020DC01092290460912F02D2
:103F1000709130028FEF0E94C82580914B0281FD85
:103F200002C090E001C091E080914B028B7F8260E3
:103F300080934B02892F0895EF92FF920F931F9366
:103F4000DF93CF9300D000D000D0CDB7DEB77C0197
:103F5000FE01319686E0DF011D928A95E9F7F701AF
:103F6000208D318D428D538D2030F8E23F07F0E0F7
:103F70004F07F0E05F072CF0D7015C968C9186FF2D
:103F80007DC02030B0E43B07B0E04B07B0E05B07FA
:103F90000CF074C0F7016281738121153105410570
:103FA000510509F45DC06115710559F18081918158
:103FB000A0E0B0E082179307A407B50741F0CB015A
:103FC000A0E0B0E082179307A407B507D1F4D701AA
:103FD0005C968C915C978E7F5C968C935C976D91D0
:103FE0007C918E010F5F1F4FC8010E94AA2680E0BE
:103FF00065E0A8010E940A27F7011382128211824C
:104000001082D7018D919C91A0E0B0E0F701208D46
:10401000318D428D538D82179307A407B50769F43C
:10402000848D91E089278B7F848FD70158961D92CC
:104030001D921D921C925B9721C081E060E00E945E
:10404000111680E00E941125BC0182E00E94D91760
:10405000F701648D6470808D918D0E94321F09C0BC
:10406000672B39F4D7015C968C915C9784605C96E1
:104070008C93F701108E118E128E138E26960FB62A
:10408000F894DEBF0FBECDBFCF91DF911F910F918E
:10409000FF90EF900895AF92BF92DF92EF92FF9260
:1040A0000F931F93DF93CF93CDB7DEB72C970FB647
:1040B000F894DEBF0FBECDBF9C015E010894A11C29
:1040C000B11C86E0D5011D928A95E9F725313105AD
:1040D00009F49AC3263131052CF52C30310509F449
:1040E0007DC12D303105ACF42A3031054CF421303E
:1040F00031050CF0E3C32115310509F493C328C43D
:104100002A30310509F40CC42B30310509F020C4E4
:10411000FEC3213131050CF0A2C22F3031050CF065
:104120000DC333C22A38310509F4F6C32B383105E3
:10413000A4F42B31310564F4293131051CF5263105
:10414000310509F41BC32731310509F001C40BC146
:104150002332310509F0FCC3F2C32F3831054CF48A
:104160002D3831050CF011C22C38310509F0F0C39F
:10417000E9C1213931050CF4FBC22739310509F0B9
:10418000E7C3E4C380914B0283FF03C010914F0249
:1041900002C010914D0200E02931310509F401E01F
:1041A000E09050020E944125FC01F7800E944125C9
:1041B000FC01808184FF35C017FD05C080E000232D
:1041C00009F481E0082F002311F001E02CC0812FB9
:1041D00090E08F779070892B79F4809143029091D1
:1041E0004402A0914502B09146020097A105B10595
:1041F00019F4212F2058ADC08091F7039091F80356
:10420000A091F903B091FA03845D9E4FAF4FBF4F69
:104210008093430290934402A0934502B0934602D8
:1042200024C0002311F10E944125FC01808185FFFB
:1042300007C080914E0283300CF08AC08F5F21C08E
:104240000E94760E833009F083C0812F90E08F7733
:1042500090702E2D30E0821793070CF079C0FEE7A6
:10426000EF16E1F5FF20E1F439C00E944125FC0181
:10427000808185FF09C080914E028E3F0CF468C09A
:10428000815080934E0264C0812F90E08F779070B0
:10429000892B09F45DC04EE7E41641F5FF2031F1AA
:1042A00081E0F81619F460E820E00EC0A2E0FA16EA
:1042B00019F46EE324E108C0B3E0FB1619F466E1DB
:1042C0002AE002C060E820E8812F90E030E000237F
:1042D00041F08F779070821793075CF4212F2F5F46
:1042E00038C08F779070281739071CF0212F215084
:1042F00030C0462F50E0812F90E08F7790704817A4
:1043000059071CF0212F2E7F04C0212F261B2C7F44
:10431000260F211719F0002319F41BC0002361F0A8
:10432000822F90E08F7790708417950714F482E0C5
:1043300001C084E0280F0DC0822F90E08F7790702D
:104340004817590714F082E001C084E0281B01C01F
:10435000212F80914B0283FF03C020934F022078CE
:1043600020934D02F3C290914B0297FF21C088E049
:10437000892780934B0283FF0EC080914D0280936A
:104380004F02807880934D0210924E0280E799E1AF
:1043900060E971E00AC080914F0280934D02109253
:1043A0004F0280E090E060E070E00E945615CEC2BF
:1043B00080914C028370813029F480E068E272E0E1
:1043C0000E94F21680914D028058807880934D02B1
:1043D00010924E0280914B02877FAEC280913102D3
:1043E00090913202009709F07DC0E0904702F09072
:1043F00048020091490210914A021E141F0410063F
:1044000011060CF06FC0D0904C028D2D0E94F51754
:1044100090E0A0E0B0E08E159F05A007B1070CF476
:1044200058C081E090E0A0E0B0E00E2C04C0880FFE
:10443000991FAA1FBB1F0A94D2F720913502309111
:104440003602409137025091380282279327A427E1
:10445000B5278093350290933602A0933702B0932C
:10446000380280914B02806880934B02E0E1EE16A7
:10447000F104010511050CF4BAC160912F0270918D
:104480003002C5010E94AA262091350230913602E1
:104490004091370250913802CA01AA27BB278F7773
:1044A0008B8377E156954795379527957A95D1F780
:1044B000822F8F778C8367E05695479537952795A0
:1044C0006A95D1F72D8380E06DE0A5010E940A274F
:1044D0008EC1F3E0DF22DF1609F038C28FE292E0EE
:1044E00061E040C160914B0267FF10C0892B71F001
:1044F0008091390290913A0221E030E0822793279F
:1045000090933A0280933902606119C0809135021C
:1045100090913602A0913702B091380221E030E04C
:1045200040E050E082279327A427B52780933502E7
:1045300090933602A0933702B09338026F7E609357
:104540004B0204C28091310290913202892B29F4EE
:1045500080914B028F7780934B0280914B0285FFB5
:10456000F5C18091470290914802A0914902B09113
:104570004A02181619061A061B060CF0F9C08FE23B
:1045800092E060E00E94A918F3C086E0FE01379631
:10459000DF011D928A95E9F78091470290914802C8
:1045A000A0914902B0914A020097A105B10509F412
:1045B00054C0893FE7E09E07E0E0AE07E0E0BE07B9
:1045C0000CF0C4C18C0101501040000F111FC90133
:1045D0008F7790700E9709F4016027FF23C01A8629
:1045E00080914B0283FD05C080E090E060E070E0C8
:1045F00004C080E799E160E971E00E94561581E00E
:1046000060E671E00E94F21682E068E671E00E94C6
:10461000F21610924702109248021092490210922C
:104620004A0202C081E08A87802F8F778F83C8017A
:10463000880F892F881F990B91958F778887812FF5
:104640008295869586958370898780E066E0AE01C5
:10465000495F5F4F0E940A2779C127FD77C1022F6A
:104660000D5010914B0217FF0AC0809131029091BA
:104670003202892B21F4213131050CF40C5F809139
:104680004C020E94F517081708F060C10430A0F032
:104690008091F7039091F803A091F903B091FA0388
:1046A0008C509E4FAF4FBF4F80933F02909340027C
:1046B000A0934102B093420217FF1DC080913102C6
:1046C00090913202892BB9F082E090E0A0E0B0E056
:1046D00004C0880F991FAA1FBB1F0A95D2F720910B
:1046E000390230913A022827392730933A02209331
:1046F0003902106120C082E090E0A0E0B0E004C088
:10470000880F991FAA1FBB1F0A95D2F72091350267
:104710003091360240913702509138028227932718
:10472000A427B5278093350290933602A0933702D1
:10473000B09338021F7E10934B0208C1809147024C
:1047400090914802A0914902B0914A020097A105B8
:10475000B10509F484CF60E02F30310509F461E040
:104760008FE292E00E94A91880914B028062E4C01F
:1047700080914B028F7D80934B0239C0809147021C
:1047800090914802A0914902B0914A020097A10578
:10479000B105B1F180914B0282FD32C00E94760ECC
:1047A000833019F580915002282F30E040E050E02E
:1047B0008091470290914802A0914902B0914A022B
:1047C000281739074A075B0744F4209347023093C0
:1047D00048024093490250934A0280914D028078EA
:1047E00090914702892B80934D0210924E021092B5
:1047F0004702109248021092490210924A02A6C043
:1048000080E060E243E00BC080914B0287FF04C070
:1048100080E060E242E003C080E060E240E00E94AD
:10482000202794C080914B0287FF12C080913302F1
:1048300090913402009709F48BC0A0E0B0E080931F
:10484000470290934802A0934902B0934A021EC0C7
:1048500082FF21C08091470290914802A0914902B5
:10486000B0914A020097A105B105A9F486E00E9423
:1048700085458091470290914802A0914902B091EC
:104880004A020097A105B10509F462C08FE292E0E7
:104890000E949C1F5DC08091470290914802A091A8
:1048A0004902B0914A020097A105B10539F48FEF92
:1048B0000E94854581E00E94541B4AC0790100276F
:1048C000F7FC0095102F609147027091480280918B
:1048D000490290914A022AE030E040E050E00E9414
:1048E000F24BE60EF71E081F191FF0E0EF16F0E876
:1048F000FF06F0E00F07F0E01F0754F5E0924702D3
:10490000F09248020093490210934A021FC08FE2BE
:1049100092E00E949C1F1AC080914B028F770CC0BE
:1049200010924702109248021092490210924A02D5
:1049300080914B028B7F806880934B0207C08091EF
:104940004D02807880934D0210924E020E94790EA3
:104950002C960FB6F894DEBF0FBECDBFCF91DF917E
:104960001F910F91FF90EF90DF90BF90AF9008954F
:104970001F93182F823118F02AEC37E032C00E94C2
:104980004125FC012581243039F0253079F0812F33
:1049900090E02130F1F414C0212F30E054E0220FD8
:1049A000331F5A95E1F7265B3C4F1BC0212F30E0A7
:1049B00044E0220F331F4A95E1F726593B4F11C0BF
:1049C0009C0194E0220F331F9A95E1F726573A4F46
:1049D00008C09C0184E0220F331F8A95E1F7265519
:1049E000394FC9011F910895882319F02FE138E04C
:1049F00016C00E944125FC018581843029F0853054
:104A000031F0813051F406C02BED37E008C02CEEB8
:104A100037E005C02DEF37E002C02EE038E0C901D5
:104A200008951F93182F833218F02BE731E126C029
:104A30000E944125FC018581843029F0853051F0A8
:104A40008130B1F40EC081E1189F90011124215DE5
:104A5000374F14C081E1189F900111242E57354F14
:104A60000DC081E1189F900111242B52334F06C0D5
:104A700081E1189F90011124285D304FC9011F91D9
:104A8000089581E692E0089590916102982309F0DB
:104A900091E0892F08952CEF3FEF41E050E04BBFAC
:104AA000F90127913791479156915070B901CA0188
:104AB00008958FEF9FEFA1E0B0E0ABBFFC018791BD
:104AC000823029F4079902C080E8089582E00895B1
:104AD000FC01848D81FD02C020E006C020E08081C1
:104AE0009181892B09F021E0822F0895FC01848DAA
:104AF00081FD02C020E006C020E082819381892BE5
:104B000009F021E0822F0895F89488E181BD8BE0BF
:104B100081BDFFCFBF92CF92DF92EF92FF920F93B2
:104B20001F93CF93DF93082F6B01EA0141155105C5
:104B300029F10E9402187C0110E086E0B82E80E086
:104B4000602FA6010E940A27B0922A0402C00E9488
:104B50007D0EC701FE010995882321F480912A0466
:104B60008823A9F70E94B626811110E0C701FE0133
:104B70000995882319F41F5F1A3008F3DF91CF914C
:104B80001F910F91FF90EF90DF90CF90BF9008950D
:104B9000DF93CF9300D000D000D0CDB7DEB7611542
:104BA000710531F14115510519F1FE01319686E08B
:104BB000DF011D928A95E9F7862F8F778983660F2B
:104BC000672F661F770B7195862F8F778A83842FC7
:104BD0008F778B83440F452F441F550B5195842F9E
:104BE0008F778C8382E0BF0146E755E20E948A25D9
:104BF00026960FB6F894DEBF0FBECDBFCF91DF91E2
:104C00000895DF93CF9300D000D000D0CDB7DEB7AA
:104C100061157105C1F0FE01319686E0DF011D923C
:104C20008A95E9F7862F8F778983660F672F661F2E
:104C3000770B7195862F8F778A8381E0BF0148E6D5
:104C400055E20E948A2526960FB6F894DEBF0FBE65
:104C5000CDBFCF91DF910895CF93DF93C0E0D0E037
:104C6000CE010E94B94EFE01EF59FD4F60818617BB
:104C700019F0CE010E94C14EA8952196C032D105EF
:104C800079F7DF91CF9108958095909161029823F3
:104C9000909361020E942C26089590916102982BB6
:104CA000909361020E942C260895809366020E94D0
:104CB0002C26089590916602973008F091E080E1EB
:104CC000E1E6F2E0DF011D928A95E9F788E1809341
:104CD0006502909366020E942C26089581E692E078
:104CE00060E070E040E250E00E94A94E80916302D3
:104CF000909164028F5F9F4F11F40E945A26809119
:104D00006602873010F0109266028AEF9FEFA1E0F2
:104D1000B0E0ABBFFC019791892F81508E3F10F41A
:104D200090936F000895FC0120E090E037E08191BE
:104D3000982780E097FF03C0990F932701C0990F30
:104D40008F5F8830B9F72F5F283089F797FD9095EE
:104D5000892F0895FC01862F8F778083660F672F38
:104D6000661F770B71956F77618308958091890233
:104D7000882319F01092890281E00895209103019F
:104D8000309104019093040180930301C9010895B7
:104D9000E0918102F0918202309709F0099508951F
:104DA0008091020108950F931F93DF93CF93CDB7A6
:104DB000DEB729970FB6F894DEBF0FBECDBFDA017C
:104DC00080910201806889836A83FE0133969E0187
:104DD000275F3F4F109721F08D918F77808301C01F
:104DE00010823196E217F307A9F78E010F5F1F4F6C
:104DF000C8010E9493268987C8010E94E81029965D
:104E00000FB6F894DEBF0FBECDBFCF91DF911F91DB
:104E10000F9108950F931F93CF93DF93082F162FB1
:104E2000EA0102C00E947D0E802F612FAE010E9418
:104E3000D3268823B9F3DF91CF911F910F91089565
:104E4000DF93CF9300D000D000D0CDB7DEB7FE0106
:104E5000319696E0DF011D929A95E9F74983AF01FB
:104E60000E940A2726960FB6F894DEBF0FBECDBF6C
:104E7000CF91DF910895FF920F931F93CF93DF930C
:104E8000082FEB014115510519F42FEF3FEF4FC0EB
:104E90008091030190910401509304014093030118
:104EA0009093820280938102109285028EEF9FEF91
:104EB0009093840280938302309388022093870228
:104EC00010E094E0F92E002361F080E0602FAE0145
:104ED0000E940A2706C00E947D0E809186028823C8
:104EE00011F0F0922A0490918502992321F4809187
:104EF0002A04882381F780918902882319F010926F
:104F0000890210E0992319F41F5F1830E0F28091B4
:104F10008102909182029093040180930301109288
:104F20008202109281022091830230918402C90191
:104F3000DF91CF911F910F91FF90089520E030E015
:104F40000E943B270895DF92EF92FF920F931F93E9
:104F5000DF93CF93CDB7DEB729970FB6F894DEBFB6
:104F60000FBECDBF8E010F5F1F4F29EEE22E28E24C
:104F7000F22EDD24D3941CC0C8010E94932699858B
:104F80008917B1F41BC0D092890212C0809103012D
:104F900090910401892B21F4F0920401E092030125
:104FA000E0910301F0910401309711F0C8010995D7
:104FB000C8010E941211892BF9F604C08A8186303B
:104FC00029F7E1CF29960FB6F894DEBF0FBECDBF0B
:104FD000CF91DF911F910F91FF90EF90DF90089597
:104FE0002F923F924F925F926F927F928F929F92F9
:104FF000AF92BF92CF92DF92EF92FF920F931F93E7
:10500000DF93CF93CDB7DEB729970FB6F894DEBF05
:105010000FBECDBF0E944B259B01AC0110E8612E55
:105020001FE3712E812C912C6222732284229522FF
:10503000B7E09594879477946794BA95D1F7A12CAB
:10504000A0ECBA2EAFE1CA2ED12CA222B322C422E8
:10505000D522FEE0D594C794B794A794FA95D1F7DA
:10506000E12CF12CE0EE0E2F112DE222F32204238D
:10507000152375E115950795F794E7947A95D1F77F
:105080006FE7262E312C412C512C22223322442230
:1050900055222DC0A8958A81843049F5CE0101960C
:1050A0000E9493269985891711F541C08D8190E062
:1050B000A0E0B0E0681679068A069B06C1F48C81F0
:1050C00090E0A0E0B0E0A816B906CA06DB0679F4C5
:1050D0008B8190E0A0E0B0E0E816F9060A071B0714
:1050E00031F489818F778093020181E007C0CE017E
:1050F00001960E941211892B69F680E029960FB65D
:10510000F894DEBF0FBECDBFCF91DF911F910F91FD
:10511000FF90EF90DF90CF90BF90AF909F908F90D7
:105120007F906F905F904F903F902F9008958E8169
:1051300090E0A0E0B0E0281639064A065B06B9F612
:10514000B5CF0F931F93DF93CF93CDB7DEB72997DA
:105150000FB6F894DEBF0FBECDBF209102012068CC
:10516000298323E02A83282F2F772B83880F892FE9
:10517000881F990B91958F778C83862F8F778D83DE
:10518000852F869586958E8367FF02C080648E8307
:10519000CA0103E0969587950A95E1F78F778F838B
:1051A000842F8295807788878E010F5F1F4FC801FB
:1051B0000E9493268987C8010E94081129960FB67C
:1051C000F894DEBF0FBECDBFCF91DF911F910F913D
:1051D0000895AF92BF92CF92DF92EF92FF920F931A
:1051E0001F93DF93CF9300D000D000D0CDB7DEB7B0
:1051F0006C010E9402185C01D60111966C91862FF9
:1052000090E0FC013397E332F10508F098C2EA5BC5
:10521000FF4FEE0FFF1F0590F491E02D0994F6016A
:1052200082810E944A0FD60117968C9184700E9449
:105230001E3285C2F50100811181D60113968C9131
:10524000139790E09695982F8827979587951296B3
:105250002C9130E0822B932B0817190709F06FC2AD
:105260000E94CE1AC8010E94AF2F69C2F601838145
:10527000E82FF0E0F695FE2FEE27F795E795D6019B
:1052800012968C91129790E0E82BF92B15968C9141
:105290001597382F330F330F20E016968C91169701
:1052A000482F50E04F77507013E0440F551F1A9568
:1052B000E1F717968C9190E08077907074E0959567
:1052C00087957A95E1F7482B592B422B532B683061
:1052D00041F4CF01BA010E94F9188091290482603B
:1052E0002FC080912904816080932904D6011796EC
:1052F0008C9180FD05C080912904826080932904EF
:10530000D60114966C91149715968C9186FD606861
:10531000CF010E94F91A0E94131811C2F60166818A
:1053200070E07695762F662777956795858190E072
:10533000682B792B84810E94111F8091290484603D
:1053400080932904E8CFD60114964C91149750E02D
:1053500015966C91159770E07695762F6627779560
:10536000679516962C911697922F9295990F990FF3
:10537000907C80E0682B792B13968C91139790E0AA
:105380009695982F88279795879512962C9130E0BF
:10539000642B752B822B932B0E940C19809129046E
:1053A0008860CECFF601628113818581E82FF0E01D
:1053B000D60116964C91169717968C911797282F11
:1053C00030E014960C91E6FD0068FE2FEE27FF0FEB
:1053D000FF0F50E04F77507083E0440F551F8A95C0
:1053E000E1F7C90180779070B4E095958795BA95FB
:1053F000E1F7482B592B812F90E09695982F88271D
:105400009795879570E04E2B5F2BE3E036952795B7
:10541000EA95E1F72170862B972B602F0E943419B3
:105420008EC1F50122A133A12115310569F0822F2A
:105430008F778983220F232F221F330B3195822FE1
:105440008F778A8318E00EC0D5018C918F7789837E
:105450008D919C91880F892F881F990B91958F773B
:105460008A8310E0F501848D80FD10610E944B2538
:10547000262F2F772B83A7E09695879577956795AD
:10548000AA95D1F7262F2F772C83F7E0969587954D
:1054900077956795FA95D1F7262F2F772D83E7E03B
:1054A0009695879577956795EA95D1F76770612B03
:1054B0006E838FEF6BE0AE014F5F5F4F0E940A2754
:1054C0003EC10E944B257B018C019B01AC012F77D3
:1054D000307040705070D60114968C9190E0A0E02E
:1054E000B0E0281739074A075B0709F05EC1A80139
:1054F000970120783F734070507067E0569547954C
:10550000379527956A95D1F7F601858190E0A0E05F
:10551000B0E0281739074A075B0709F046C1A80120
:1055200097012070307C4F7150709EE056954795E2
:10553000379527959A95D1F7868190E0A0E0B0E065
:10554000281739074A075B0709F02FC1278180E038
:1055500090E0A0EEB0E0E822F9220A231B2385E1C7
:1055600016950795F794E7948A95D1F7822F90E0E6
:10557000A0E0B0E087709070A070B070E816F906F7
:105580000A071B0709F011C18381682F70E0769527
:10559000762F662777956795828190E0682B792B27
:1055A0006115710509F401C1269526952695122FDE
:1055B00020FF0BC0A5014C5D5F4FCB0160E070E0A8
:1055C0000E944F2DBC01009721F0809102010E94A2
:1055D0000126D5018D919C911197892B09F4E5C085
:1055E00011FFE3C05C968C915C9781605C968C9314
:1055F000DCC0F601838190E09695982F88279795D7
:105600008795228130E0822B932B90932C048093FA
:105610002B0495C0D60113968C91139790E0969524
:10562000982F88279795879512962C91129730E09E
:10563000822B932B90932F0480932E0414968C919D
:10564000149780933C0415968C91159780933004A1
:1056500016968C918093310480912D04816012C044
:1056600022E030E0F601E20FF31F8081F901E05DF6
:10567000FB4F80832F5F3F4F2730310599F7809193
:105680002D04826080932D045AC0F601828180939C
:105690003704838180933804848180933904858121
:1056A00080933A0480912D048460ECCFD601159646
:1056B0008C911597882309F442C013968C91139707
:1056C000482F50E05695542F4427579547951496E8
:1056D0002C911497922F9295990F990F907C80E0BE
:1056E000482B592B12968C9190E0482B592B40FD5A
:1056F00002C067E601C062E7CA01969587950E94DD
:10570000EA2F1DC00E948425F60182810E94F418B0
:1057100016C0D60112968C91882329F00E9441254B
:10572000FC01848101C080E00E948E1508C090E0D9
:10573000D60112968C91811191E090938602F60128
:10574000208130E02F7730708091020190E028179F
:10575000390749F480912A04882329F080912A048A
:10576000815080932A04D5015C968C9181FD06C0FE
:1057700080E090E060E040E050E015C084FF09C0A8
:10578000F50182819381009721F042855385668DD2
:105790000AC0D50116964D915C9117978D919C91F9
:1057A00011975E966C910E94A12826960FB6F894E8
:1057B000DEBF0FBECDBFCF91DF911F910F91FF9044
:1057C000EF90DF90CF90BF90AF90089590938402B8
:1057D0008093830220918702309188022115310540
:1057E00049F06115710531F04115510519F0C901F4
:1057F0000E943A4C81E080938502089560E070E059
:1058000040E050E00E94E62B0895DF93CF9300D054
:1058100000D000D0CDB7DEB7FE01319626E0DF0123
:105820001D922A95E9F7282F2F772983880F892F32
:10583000881F990B91958F778A838FEF63E1AF0172
:105840000E940A2726960FB6F894DEBF0FBECDBF82
:10585000CF91DF910895DF92EF92FF920F931F9304
:10586000DF93CF9300D000D000D0CDB7DEB7E62EC7
:10587000FE01319626E0DF011D922A95E9F7282FD7
:105880002F772983880F892F881F990B91958F7700
:105890008A838FEF9FEF90932C0480932B0410E06A
:1058A000FE2E0F2F35E0D32E16C08FEF6E2D4F2D0D
:1058B000502F0E940A27D0922A0402C00E947D0E17
:1058C00080912B0490912C0497FF04C080912A04AE
:1058D0008823A1F71F5F80912B0490912C0497FFE0
:1058E00002C01A3011F720912B0430912C04C90109
:1058F00026960FB6F894DEBF0FBECDBFCF91DF91D5
:105900001F910F91FF90EF90DF90089562E10E9448
:105910002B2C089561E10E942B2C08958F929F9269
:10592000AF92BF92CF92DF92EF92FF920F931F93AD
:10593000DF93CF9300D000D000D0CDB7DEB7FC010D
:1059400079016115710509F48AC02115310509F441
:1059500086C06E010894C11CD11C86E0D6011D9240
:105960008A95E9F7CB01880F892F881F990B9195AC
:10597000BFE79B2E982214E1AFE7AA2EA6227FE76D
:10598000B72EB42265E0862E8E2F8F778983EE0F97
:10599000EF2FEE1FFF0BF1958E2F8F778A83163135
:1059A00071F0173128F4143171F0153131F505C05B
:1059B000173139F0183109F50AC090E00CC080E0C9
:1059C00008C080E005C0AB829C82BD8216C083E027
:1059D0008D5F982F9D5FF701E90FF11D80818B830B
:1059E000892F8F5FF701E80FF11D90819C838F5FF6
:1059F000F701E80FF11D80818D8310922C04109225
:105A00002B0400E015C08FEF612FA6010E940A272A
:105A100080922A0402C00E947D0E80912B049091F6
:105A20002C04892B21F480912A048823A1F70F5F8D
:105A300080912B0490912C04892B11F40A3019F7D2
:105A400080912B0490912C04892B49F0E0912B0438
:105A5000F0912C041F5F193109F096CF02C0E0E0ED
:105A6000F0E0CF0126960FB6F894DEBF0FBECDBF93
:105A7000CF91DF911F910F91FF90EF90DF90CF902A
:105A8000BF90AF909F908F900895FC01A62F9A0130
:105A900080E090E0BF014A2F0E948E2C0895AF92C3
:105AA000BF92CF92DF92EF92FF920F931F93DF93FB
:105AB000CF9300D000D000D0CDB7DEB79C018B01D2
:105AC0007A0101978F5F934008F06CC0FE01319618
:105AD00086E0DF011D928A95E9F7822F8F7789830F
:105AE000220F232F221F330B3195822F8F778A832A
:105AF00010922D04DD24BE2ECF2E8FE0A82E1EC0C6
:105B00008FEF60E14B2D5C2D0E940A27A0922A04A2
:105B100002C00E947D0E80912D04873021F080917B
:105B20002A048823B1F780912D04873031F082B7A1
:105B300090E08C599F4F0E949412D39480912D0431
:105B4000873019F0BAE0DB16D9F680912D04873042
:105B500021F4809130048F3759F40115110511F0AB
:105B6000F8011082E114F104E9F0D7011C921AC087
:105B70000115110521F080913C04F8018083E114A6
:105B8000F10459F0D701E0E3F4E08BE001900D92CD
:105B90008150E1F7D7011B961C9220912E04309181
:105BA0002F0402C020E030E0C90126960FB6F89419
:105BB000DEBF0FBECDBFCF91DF911F910F91FF9040
:105BC000EF90DF90CF90BF90AF90089510923E0479
:105BD00090913E0490933D0490913D049093600415
:105BE0009091600490935F04119A1098199A1898F4
:105BF00092E09BB9883008F087E0E82FF0E0EE0FE4
:105C0000FF1FE857FE4EA591B491653010F465E092
:105C100003C0693008F068E04F7D6550660F453479
:105C200011F4606203C04F3409F46063223008F05D
:105C300068608B2F992787FD9A958F7080939000CD
:105C4000A9B96093950088EB8AB980E090E0089547
:105C50001F920F920FB60F920BB60F9211248F93D3
:105C60009F93EF93FF9390915F0480916004981746
:105C700011F4559812C0E0916004F0E0E35CFB4F32
:105C800084A18CB9809160048F5F809360048091BF
:105C90006004803210F010926004FF91EF919F91A8
:105CA0008F910F900BBE0F900FBE0F901F90189505
:105CB0001F920F920FB60F920BB60F9211242F93D3
:105CC0003F938F939F93EF93FF9320913D04809197
:105CD0003E0430E090E001972817390741F08091A9
:105CE0003D048F3179F480913E04882359F48091EA
:105CF0003E048F5F80933E0480913E04803210F01A
:105D000010923E04E0913D04F0E08CB1E35CFB4F67
:105D1000828380913D048F5F80933D0480913D0498
:105D2000803210F010923D04FF91EF919F918F917E
:105D30003F912F910F900BBE0F900FBE0F901F90B1
:105D4000189527E0813D9207C0F12FE0813A920734
:105D500010F481E01EC023E28932920710F482E041
:105D600018C026E3813B920710F483E012C026E4BA
:105D70008135920710F484E00CC028E8893B920733
:105D800010F485E006C0895D964D10F087E001C0F3
:105D900086E0789420E030E05E9902C020E030E0B8
:105DA0002F5F3F4FA89597E220313907A8F368E0AD
:105DB0004EE421E00E94E62D089580E0EACF833092
:105DC000C9F0843028F4813061F0823080F40CC056
:105DD0008530B1F0853088F08630A9F08730C9F47D
:105DE00015C020E639E017C020EB34E014C020ECE9
:105DF00032E111C020E835E20EC020E438E30BC0E8
:105E000020E03BE408C020E036E905C020E031EEA8
:105E100002C020E030E0C901089539B1209190001E
:105E2000922F80E0232F30E0282B392B48E851E1D6
:105E300060E0FA01859194918217930729F06F5FD2
:105E40004E5F5F4F6830A9F7862F0E94DF2E0895BE
:105E5000482FA89503C0559A7894A89520915F047F
:105E60008091600430E090E001972817390799F39A
:105E700080915F048F3121F480916004882359F36D
:105E8000E0915F04F0E0E35CFB4F44A39FB7F8941C
:105E900080915F048F5F80935F0480915F04803204
:105EA00010F010925F049FBF559A80E090E0089533
:105EB00090913D0480913E04981719F42FEF3FEF25
:105EC00015C0E0913E04F0E0E35CFB4F9281F89452
:105ED00080913E048F5F80933E0480913E04803227
:105EE00010F010923E04292F30E07894C9010895F3
:105EF000CF92DF92EF92FF920F931F93CF93DF9396
:105F0000E82E162F042FF52E6AEC0E9406178E2D10
:105F1000612F0E940617802F9F2DEC0185E0C82E6F
:105F2000D12CCC0EDD1E0FC01881812F8A5C8430ED
:105F300028F48E2D6BEC0E9406171F708E2D612F9A
:105F40000E9406172196CC15DD0571F7DF91CF91E0
:105F50001F910F91FF90EF90DF90CF900895DF9306
:105F6000CF9300D000D000D0CDB7DEB7FE01319680
:105F700026E0DF011D922A95E9F799838A8380E064
:105F800063E0AF010E94782F26960FB6F894DEBF2B
:105F90000FBECDBFCF91DF910895DF93CF9300D097
:105FA00000D000D0CDB7DEB7FE01319696E0DF011C
:105FB0001D929A95E9F7898380E062E0AF010E9423
:105FC000782F26960FB6F894DEBF0FBECDBFCF91C7
:105FD000DF910895DF93CF9300D000D000D0CDB7EC
:105FE000DEB7FE01319626E0DF011D922A95E9F722
:105FF00099838A836F776B8380E066E0AF010E94AC
:10600000782F26960FB6F894DEBF0FBECDBFCF9186
:10601000DF910895EF92FF920F931F93DF93CF9339
:10602000CDB7DEB762970FB6F894DEBF0FBECDBF17
:10603000162F882309F094C1809194028823B1F02F
:1060400060918A0270918B0280918C0290918D02F6
:106050006C5E7F4F8F4F9F4F0E94E911882331F074
:106060001092940210929502109296028091F7037A
:106070009091F803A091F903B091FA0380938A02FA
:1060800090938B02A0938C02B0938D021A3C41F442
:10609000109294021092950281E08093960260C162
:1060A00080919602882309F45BC11B3C21F481E0B6
:1060B0008093950255C1809195028111106C1092C8
:1060C000950280919402E82FF0E0E657FD4F14838B
:1060D0008F5F80939402863008F442C10E940218B8
:1060E0008C0190918E02933009F4B4C0943030F456
:1060F000913059F1923008F055C00AC0953009F43A
:10610000C5C0953008F4B4C0963009F01FC1E8C08E
:1061100080E06CEC0E940617D80116968D919C9138
:1061200017979C012E7F3F773695279580FD306825
:10613000F801868D8F83388729870E94760E8A879B
:106140001C861B8680E060E027C080E06CEC0E942B
:106150000617D80111968C9111978F835C915D96EB
:106160004C915D97242F30E02370307094968C9181
:10617000992787FD9095282B392B232B11F480E04C
:1061800001C080E858878987842F0E94EB178A878F
:106190001C861B8680E061E0AE01495F5F4F0E9474
:1061A000782FD8C090918F0280E020919002BC019E
:1061B000620F711D9091920280E020919302820FF4
:1061C000911DAC01440F551F4E7F5F7797FD4160D5
:1061D0006115710519F4F80160817181F0E4603096
:1061E0007F0708F0B3C0D8018D919C91681779079B
:1061F00039F4CB016091910220E00E9434196DC006
:10620000862F8F778983660F672F661F770B7195AF
:10621000862F8F778A8390919102892F8F778B8336
:10622000852F869586958C8397FF02C080648C832A
:10623000CA0133E0969587953A95E1F78F778D837C
:10624000842F829580778E8380E063E0AE014F5F7C
:106250005F4F41C090918F0280E020919002820FA9
:10626000911D60E00E94321F882309F46FC035C081
:1062700040918F02442329F0842F8250823008F00D
:1062800065C080E060E20E94202727C030918F0225
:1062900020E080919002280F311DFE01319686E0AA
:1062A000DF011D928A95E9F7822F8F778983C901D3
:1062B000880F892F881F990B91958F778A83832F59
:1062C00082958695869583708B83809191028C83CD
:1062D00080E066E0AF010E940A2780E06CEC38C0E5
:1062E00030918F0220E080919002280F311D8E01A5
:1062F000035F1F4FF80111929A95E9F7F22EE32EF2
:10630000C801B9010E94AA2689E1B8014DEB51E309
:106310000E949E278C018235910569F08335910595
:1063200024F48734910591F406C08736910519F05D
:106330008237910559F480E06CEC0E940617602FBB
:106340006F778F2D9E2D0E94EA2F04C080E06DECA8
:106350000E940617109294021092950210929602D3
:1063600062960FB6F894DEBF0FBECDBFCF91DF911E
:106370001F910F91FF90EF900895FC018181893169
:1063800021F0CF010E94C8260895848190E00E94E8
:10639000FE2B0895FB0157FD02C021E004C050957B
:1063A00041955F4F20E08330910541F184309105A4
:1063B00034F48130910501F1029751F523C0843006
:1063C000910519F0059721F50AC081818F5F8183BE
:1063D00090E084179507E4F0222351F00DC08181ED
:1063E0008150818390E08417950794F0222321F057
:1063F000842F815081830CC011820AC012821382C3
:10640000168A06C090E08281882309F491E0928385
:1064100080E090E008958230910519F0039751F4DF
:1064200003C02FEF3FEF08C083E090E040E050E072
:106430000E94CA3120E030E0C90108951F93182F4F
:106440000E940218FC01848D112311F0806401C0A8
:106450008F7B848F1F9108951F93CF93DF93EC015F
:106460008A81882309F470C081E060E00E941116DF
:1064700000D000D00F92EDB7FEB7319612E0ADB765
:10648000BEB711961C9384E092E1928381838C8144
:106490009D81948383830E947F170F900F900F90AC
:1064A0000F900F908B81843079F400D00F92EDB76C
:1064B000FEB7118380E092E1938382830E947F176D
:1064C0000F900F900F9018C000D000D00F92EDB732
:1064D000FEB73196ADB7BEB711961C938CEF91E124
:1064E000928381838885838314820E947F170F9013
:1064F0000F900F900F900F90898D9A8D97FD04C08B
:1065000082E064EF71E10CC08E5F9F4F21F482E066
:106510006CEE71E105C084E00E941125BC0182E0AF
:106520000E94D91781E0888F8E8B8B81813058F043
:10653000833020F08450823030F402C083E001C008
:1065400088E08F8B01C01E8ADF91CF911F91089543
:106550009C01FB018130910569F0823091051CF4AA
:106560000097D9F027C083309105F1F0853091056F
:1065700009F517C08EEF9FEF928F818F4091A60291
:106580005091A702CA0101978050944018F4558396
:10659000448310C0358324830DC0CB010E942C326C
:1065A00009C081E0838306C083E090E040E050E0D2
:1065B0000E94CA3180E090E008951F93182F81E077
:1065C00060E00E941116113049F0113028F01230AD
:1065D00039F0133071F406C083E105C084E103C0D3
:1065E00085E101C086E10E941125BC0182E00E9484
:1065F000D9171F9108951F93CF93DF93EB0182303A
:10660000910509F493C0833091051CF4892B31F076
:10661000BBC0863091050CF0B7C075C081E060E06A
:106620000E9411168A818823A1F000D000D00F9219
:10663000EDB7FEB7319682E0ADB7BEB711968C9339
:1066400086EB91E1928381838C819D819483838306
:1066500046C0209197023091980240919902509142
:106660009A02211531054105510509F440C08DB745
:106670009EB707970FB6F8949EBF0FBE8DBFEDB7BC
:10668000FEB7319612E0ADB7BEB711961C938EEAF5
:1066900091E19283818323833483458356830E94CF
:1066A0007F176C817D818DB79EB707960FB6F894E2
:1066B0009EBF0FBE8DBF6115710509F465C000D086
:1066C00000D00F92EDB7FEB73196ADB7BEB71196B9
:1066D0001C9389EA91E192838183748363830E948E
:1066E0007F170F900F900F900F900F904DC08C81DF
:1066F0009D8197FF49C084E00E941125BC0182E082
:106700000E94D91741C08330910551F4109297022D
:10671000109298021092990210929A021D821C8285
:10672000BE0142E050E00E94CA312EC08A81882317
:1067300071F41D821C8283E08B838FEF9FE39F8324
:106740008E8391E0988F85E08F8B9E8B17C01E8A79
:106750008C819D810E944A4A6093970270939802AF
:106760008093990290939A021B82611571058105AD
:10677000910521F48FEF9FEF9D838C8390E08A81B8
:10678000882309F491E09A8380E090E0DF91CF9133
:106790001F910895FF920F931F93CF93DF93EC0106
:1067A0008B01F42E0E944125FC01C230D10509F471
:1067B0008BC0C330D10534F42097D1F0219709F074
:1067C0009BC00DC0C430D10509F463C0C430D105ED
:1067D0000CF463C0C530D10509F08EC05EC0FF2047
:1067E00019F08485D8016DC08385F801818384C048
:1067F00081E060E00E941116FF2059F1D801119646
:106800002C91EDB7FEB737970FB6F894FEBF0FBEC9
:10681000EDBF319682E0ADB7BEB711968C9381EC97
:1068200091E192838183822F6AE00E94114C8383DD
:106830001482822F0E94114C958316820E947F172A
:10684000EDB7FEB737960FB6F894FEBF0FBEEDBF9B
:1068500053C000D000D00F92EDB7FEB7319682E062
:10686000ADB7BEB711968C938BEB91E19283818388
:10687000D80111968C9122E3829FC0011124948348
:1068800083830E947F170F900F900F900F900F90AF
:1068900033C0F80181818F3F79F1FF2019F44BEE6D
:1068A0005FEF02C040E05FEFCE01B8010E94CA3145
:1068B000FF2011F1D80111968C9111978823E1F4F2
:1068C00081E011968C9318C0D80112968C91129782
:1068D000882349F011968C91FF2011F0848701C024
:1068E00083870E942C2690E0F8018281882309F496
:1068F00091E0D80112969C9380E090E0DF91CF91D7
:106900001F910F91FF90089541E00E94CA330895AE
:1069100040E00E94CA3308951F93CF93DF93EB01A9
:1069200082309105C1F18330910534F40097C1F0B4
:10693000019709F04CC005C0863091050CF047C0A6
:1069400025C00E944125FC01808185FF02C082E0B4
:1069500003C084FF03C081E0898339C0198237C036
:1069600081E060E00E9411168981825F0E941125FA
:1069700000D00F9222E0EDB7FEB72183938382838C
:106980000E947F170F900F900F9021C043E050E0BE
:106990000E94CA311CC08A81882399F00E94412537
:1069A000FC0110811F7C8981813011F4106103C0CA
:1069B000823009F410620E944125FC0110830E947C
:1069C0002C2690E08A81882309F491E09A8380E064
:1069D00090E0DF91CF911F910895CF93DF93EB016A
:1069E0008230910581F1833091052CF4009781F07C
:1069F0000197C9F504C086309105ACF51FC00E940F
:106A00004125FC0187818983843068F119822BC07C
:106A100081E060E00E9411168981865F0E94112545
:106A200000D00F9222E0EDB7FEB7218393838283DB
:106A30000E947F170F900F900F9015C044E050E018
:106A40000E94CA3110C08A81882339F00E944125F2
:106A50002981FC0127830E942C2690E08A818823CB
:106A600009F491E09A8380E090E0DF91CF9108955E
:106A70001F93CF93DF939C01EB018230910509F4C2
:106A800084C0833091053CF4009749F18130910531
:106A900009F0AEC005C0863091050CF0A9C070C0E9
:106AA0008C819D8101978C5F934010F03D832C83F6
:106AB0008CEF93E09F838E8311E01B831E8B83E01A
:106AC0008F8B188F8C819D810197880F991F0E9451
:106AD0003B481982039709F08BC0198389C081E074
:106AE00060E00E9411168B81813079F52C813D8107
:106AF0008DB79EB707970FB6F8949EBF0FBE8DBF98
:106B0000EDB7FEB7319682E0ADB7BEB711968C9364
:106B100085E091E092838183348323832D5F3F4F0F
:106B2000368325830E94AC178DB79EB707960FB6A4
:106B3000F8949EBF0FBE8DBF89818C5F0E94B824E0
:106B4000BC0182E00E94D91753C000D000D00F9240
:106B5000EDB7FEB7319682E0ADB7BEB711968C9314
:106B60008FE091E0928381838C819D8194838383E4
:106B70000E94AC170F900F900F900F900F9038C09D
:106B800042E050E00E94CA3133C08A81882399F0E4
:106B90002C813D818981882319F461E070E002C075
:106BA00063E070E021503040C901880F991F0E94B6
:106BB00010481A821DC08B81813019F48A831E8A85
:106BC00017C08C819D8101978C7F01969D838C835A
:106BD0000197880F991F0E943B481982039711F46F
:106BE00081E0898391E09B839E8B83E08F8B988FDC
:106BF00080E090E0DF91CF911F910895CF93DF93D4
:106C0000EB018230910541F1833091052CF400971E
:106C100089F00197E9F504C086309105CCF517C0DD
:106C200080E090E00E943B481982039789F581E05B
:106C300089832EC081E060E00E94111689818E5FF9
:106C40000E94B824BC0182E00E94D91721C042E012
:106C500050E00E94CA311CC08A81882399F081E0EB
:106C600060E00E94111682E069EC71E10E94D91780
:106C70008981882319F481E090E002C083E090E0EC
:106C80000E94EC4790E08A81882309F491E09A837E
:106C900080E090E0DF91CF910895CF93DF93EB01F7
:106CA0008230910509F450C08330910534F4009787
:106CB00069F0019709F054C005C0863091050CF0C9
:106CC0004FC03DC00E94394989834AC081E060E0DD
:106CD0000E94111669816623A9F48CE10E94112596
:106CE00000D00F9222E0ADB7BEB711962C9311974A
:106CF00013969C938E9312970E947F170F900F907C
:106D00000F902EC000D000D00F92EDB7FEB7319695
:106D100082E0ADB7BEB711968C9388ED91E1928376
:106D2000818385E0689FC0011124948383830E943E
:106D30007F170F900F900F900F900F9011C049EC9C
:106D400050E00E94CA310CC08A81882319F08981E1
:106D50000E94114990E08A81882309F491E09A8386
:106D600080E090E0DF91CF9108951F93CF93DF9360
:106D7000EB01122F8230910519F1833091052CF42B
:106D8000009761F0019779F504C0863091055CF5B4
:106D900012C0842F0E94224B898325C081E060E0CD
:106DA0000E9411168981810F0E94B824BC0182E0E3
:106DB0000E94D91718C042E050E00E94CA3113C0A7
:106DC0008A81882351F08981882321F0842F0E94B1
:106DD000824B03C0842F0E94564B90E08A81882307
:106DE00009F491E09A8380E090E0DF91CF911F91C8
:106DF000089544E026E00E94B536089541E020E081
:106E00000E94B536089548E022E00E94B536089504
:106E1000CF93DF93EB018130910569F082309105CA
:106E20001CF4892B69F04CC08230910579F10397ED
:106E300009F046C024C00E94F0489D838C8340C066
:106E400081E060E00E94111600D000D00F92EDB7F3
:106E5000FEB7319682E0ADB7BEB711968C938EED3A
:106E600091E1928381838C819D81948383830E94AD
:106E70007F170F900F900F900F900F9021C083E01D
:106E800090E040E050E00E94CA311AC08A81882315
:106E900061F483E08B8384E390E09F838E8391E0B1
:106EA000988F82E08F8B9E8B05C01E8A8C819D817E
:106EB0000E94CF4890E08A81882309F491E09A8368
:106EC00080E090E0DF91CF910895CF93DF93EB01C5
:106ED0008230910581F18330910534F40097C9F037
:106EE000019709F044C005C0863091050CF03FC001
:106EF0001DC00E944B46813051F0813018F0833024
:106F000029F402C0198233C082E001C083E0898382
:106F10002EC081E060E00E9411168981885F0E9486
:106F2000B824BC0182E00E94D91721C044E050E09F
:106F30000E94CA311CC08A81882399F089818130DE
:106F400049F0813028F0823039F0833051F406C0A6
:106F500080E005C081E003C083E001C087E00E94BB
:106F6000114690E08A81882309F491E09A8380E0B9
:106F700090E0DF91CF910895CF93DF93EB018230C2
:106F8000910549F1833091051CF4892B29F02EC01D
:106F9000863091055CF51AC08A81882339F180E03A
:106FA00061E00E94111681E20E941125BC0182E07D
:106FB0000E94D91781E060E00E94111689E10E94C9
:106FC0001125BC0182E00E94D91710C040E050E0BA
:106FD0000E94CA310BC08A81882311F00E9459494E
:106FE00090E08A81882309F491E09A8380E090E020
:106FF000DF91CF9108950F931F93CF93DF93FC01FF
:107000008B01EA0180819181892B21F0858D83702C
:10701000833081F081E060E00E94111685E00E94DB
:107020001125BC0182E00E94D91780E003301105D0
:1070300041F526C00E94760E833011F10E94760E33
:107040008230F1F00630110559F480E060E243E04F
:107050000E94202781E090E0BE010E94A8320EC06D
:1070600081E060E00E94111686E00E941125BC01BB
:1070700082E00E94D9171A821B821E8A80E001C01A
:1070800081E0DF91CF911F910F910895EF92FF92D0
:107090000F931F93CF93DF938C01EB010E94021893
:1070A0007C01B801AE010E94FB37882309F4B1C00E
:1070B0000230110509F491C00330110544F40115A3
:1070C000110549F10130110509F0A3C00DC00430CC
:1070D000110509F45EC0043011050CF476C00530CA
:1070E000110509F096C062C08EEF9FEF9A8F898FCD
:1070F0002091A6023091A702C901019780509440C7
:1071000018F43D832C8302C01D830C8380E094E03F
:107110009F838E837EC08A81882309F47AC081E0B0
:1071200060E00E9411162C813D8137FF14C000D011
:107130000F9282E0ADB7BEB711968C93119787EE90
:1071400091E113969C938E9312970E947F170F9054
:107150000F900F9018C000D000D00F92EDB7FEB77F
:10716000319682E0ADB7BEB711968C9383EE91E174
:1071700092838183348323830E947F170F900F9023
:107180000F900F900F9083E08F8B81E0888F8E8B14
:1071900040C08C819D8101969D838C832E813F818F
:1071A000821793077CF03D832C830CC08C819D81DA
:1071B00001979D838C831816190624F081E090E0D6
:1071C0009D838C8381E08B8324C083E090E0BE01AB
:1071D00040E050E00E94CA311CC091E09B838A814C
:1071E0008823B1F02C813D811216130694F42150AE
:1071F0003040F7018081918160E041E000E00E9431
:1072000069468C819D819093A7028093A60201C05C
:107210009A8380E090E0DF91CF911F910F91FF90D2
:10722000EF9008950F931F93CF93DF93EC01062FF8
:10723000142F8A818823F9F481E08B83643019F458
:1072400088E090E002C080E094E09F838E832C81F0
:107250003D818E819F818217930724F481E090E025
:107260009D838C8381E08A83083009F4E0C080E04C
:107270000E944A0FDCC08C819D819093A70280936D
:10728000A602643009F1653060F4613009F49EC0F3
:107290006130D0F0623009F49BC0633009F0C7C0A0
:1072A000C4C0673009F492C0683038F4653009F41E
:1072B0008DC0663009F0BBC007C0683009F467C0F4
:1072C000693009F0B4C082C08B818150823080F572
:1072D0008EEF9FEF9A8F898FCE010E942C3281E032
:1072E0006AE00E94111681E10E941125BC0182E032
:1072F0000E94D917043051F0063069F0002391F450
:107300008C819D8101970E9441470AC08C818150E8
:107310000E946E4705C08C819D8101970E943C4769
:107320009A8F898F898D9A8D97FD56C0888754C012
:1073300081E06AE00E94111682E10E941125BC01E1
:1073400082E00E94D917043061F00630B9F00023C2
:1073500009F042C08C819D81019768850E940D478C
:1073600013C08C819D81893091051CF08FEF9FEFB8
:107370000BC0815068850E94464706C08C819D8164
:10738000019768850E9406479A8F898F25C00E94C1
:107390000218FC014081518141155105E9F0858DAC
:1073A00083708330C9F42C813D8121153105A1F012
:1073B0008B818150823080F021503040CA01612F92
:1073C00040E008850E9469461B8231C084E02EC0DF
:1073D0008B818150823010F481E028C081E06AE026
:1073E0000E9411168B81863071F481E10E94112573
:1073F000BC0182E00E94D9178C819D81019769852B
:107400000E94C1470EC082E10E941125BC0182E0AA
:107410000E94D9178C819D8101976985498D0E94B1
:107420008F479A8F898F86E001C087E08B83DF9139
:10743000CF911F910F9108950F931F93CF93DF93D7
:10744000EC018B010E940218BE01A8010E94FB37CB
:107450008823F1F0C230D10549F0C430D105A1F440
:10746000C80169E040E00E94123912C0C80168E01A
:1074700040E00E941239F8018381882349F40E9478
:107480000D162FEF3FEF06C0CE01B8010E94A832C3
:1074900020E030E0C901DF91CF911F910F91089555
:1074A0008230910531F08430910549F4CB0167E0D9
:1074B00002C0CB0166E040E00E94123902C00E9487
:1074C000A83280E090E008958230910531F0843058
:1074D000910549F4CB0165E002C0CB0164E040E0D6
:1074E0000E94123902C00E94A83280E090E0089504
:1074F0008230910531F08430910549F4CB0161E08F
:1075000002C0CB0160E040E00E94123902C00E943C
:10751000A83280E090E008951F93182F1816B4F455
:1075200080E00E94DD3280E090E0612F0E940D47F4
:10753000892B39F48CE190E065E040E00E948F47B0
:1075400007C0812F0E94B146892B11F082E001C053
:1075500083E00E94DD3284EF91E00E9494121F913B
:107560000895CF92DF92EF92FF920F931F93CF93E4
:10757000DF937B018130910571F0823091051CF41D
:10758000892B89F0D0C08230910509F452C003974D
:1075900009F0C9C047C08FEF9FEFDB0115969C93A0
:1075A0008E931497C0C0FB018281882309F4BBC06D
:1075B00081E060E00E941116D70114962D913C9154
:1075C000159737FF10C000D00F9282E0EDB7FEB7DD
:1075D00081838EE092E1938382830E947F170F90D4
:1075E0000F900F9018C000D000D00F92EDB7FEB7EB
:1075F000319682E0ADB7BEB711968C938AE092E1E6
:1076000092838183348323830E947F170F900F908E
:107610000F900F900F9085E0F701878B81E0808FAE
:10762000868B81C083E090E040E050E00E94CA3148
:107630007AC0DB0112968C911297882399F11496E7
:10764000CD91DC911597C038D10520F48C2F0E9484
:107650008C3A2FC0B0E4C030DB0708F06FC080E088
:107660000E94DD326E016D2D606C80E190E00E9421
:107670000D47892B09F062C081E190E06C2F0E94D8
:107680000D47892B09F05AC08CE190E065E041E09C
:107690000E948F4783E00E94DD3284EF91E00E94D8
:1076A000941207C081E00E94DD3281E0D70112967A
:1076B0008C93F7018481958101978F37910550F460
:1076C00080E090E00E944147D70115969C938E93ED
:1076D000149715C080E190E00E944147182F00E008
:1076E000F7011583048381E190E00E944147082B54
:1076F000192B1F73D70115961C930E931497F7013E
:1077000084819581805098423CF08FEF9FEFD701A4
:1077100015969C938E93149781E0F70183838FEFE6
:1077200097E29783868380E090E0DF91CF911F916D
:107730000F91FF90EF90DF90CF90089582E0ABCF54
:10774000CF93DF93EB018230910509F44CC0833075
:10775000910509F441C0892B09F05DC08A81882315
:1077600009F459C081E060E00E9411162C813D812E
:1077700037FF14C000D00F9282E0ADB7BEB71196AC
:107780008C93119789E192E113969C938E931297B3
:107790000E947F170F900F900F9018C000D000D05C
:1077A0000F92EDB7FEB7319682E0ADB7BEB7119636
:1077B0008C9385E192E192838183348323830E94B9
:1077C0007F170F900F900F900F900F9083E08F8B8B
:1077D00081E0888F8E8B1FC083E090E040E050E016
:1077E0000E94CA3118C08A81882321F08C810E94AE
:1077F0008C3A05C081E00E94DD3281E08A8380E01E
:1078000090E00E9441479D838C8381E08B838FE7CA
:1078100090E09F838E8380E090E0DF91CF91089588
:10782000CF93DF93EB018230910509F48FC0833051
:10783000910534F40097B1F0019709F08CC00CC0A9
:107840008430910509F46DC0843091050CF477C043
:10785000059709F080C06BC081E090E00E94A832DB
:10786000198679C08A81882309F475C081E060E0B7
:107870000E9411168B81882331F482E06DE272E15F
:107880000E94D91725C08DB79EB707970FB6F894F9
:107890009EBF0FBE8DBFEDB7FEB7319682E0ADB78C
:1078A000BEB711968C938EE192E1928381838C8195
:1078B0009D81948383838985858316820E947F17A7
:1078C0008DB79EB707960FB6F8949EBF0FBE8DBFBB
:1078D000898D9A8D97FD0AC0823091051CF0029720
:1078E00029F402C0805D03C08FE301C085E40E94DB
:1078F000CE1581E0888F8E8B8B81863059F0873052
:1079000020F48150823058F403C0873041F404C021
:1079100086E003C08CE001C08EE08F8B1CC01E8A05
:107920001AC08B81863041F4CB0163E011C08B819A
:10793000863011F481E001C086E08B830CC083E0C7
:1079400090E040E050E00E94CA3105C0CB0162E007
:1079500040E00E94123980E090E0DF91CF910895DD
:10796000AF92BF92CF92DF92EF92FF920F931F934D
:10797000CF93DF938C01EB018230910509F491C024
:10798000833091053CF4009771F08130910509F046
:10799000A1C05DC08330910509F455C086309105C2
:1079A0000CF098C06CC08A81882309F493C0809140
:1079B0009B02882309F48EC081E060E00E941116CA
:1079C00000D000D00F92EDB7FEB7319682E0ADB790
:1079D000BEB711968C9382E093E1928381838C8170
:1079E0009D81948383830E947F170F900F900F9047
:1079F0000F900F9089810E94AE485C01C12CE0E895
:107A0000DE2E70E8E72EF12C00E010E0C6018A219E
:107A10009B21892B11F424E001C026E0C7018A21B3
:107A20009B21892B09F02F5F822F0E94CE15F6949F
:107A3000E7940F5F1F4F0830110519F0D694C794D3
:107A4000E5CF1E8A47C01E8A81E00E9466480E94D8
:107A5000F04880939B0284E068E072E00E94F21696
:107A600085E060E172E00E94F21686E068E172E073
:107A70000E94F21687E060E272E00E94F2164091E6
:107A80009B02C801BE0150E00E94CA31898190E08A
:107A900001969D838C838B818230E1F488E08B8317
:107AA00019C08A81882389F481E090E09D838C83CA
:107AB00080919B028E831F8211E01A8380E00E94D6
:107AC0006648188F85E08F8B1E8B88E08B838C81B6
:107AD0008150898380E090E0DF91CF911F910F91D9
:107AE000FF90EF90DF90CF90BF90AF9008951F93DD
:107AF00080919D02803178F010929D0210929C023C
:107B000081E061E00E94111610E085EA0E94CE1526
:107B10001F5F1F30D1F781E060919D020E94111616
:107B200080919C02813039F0813018F0823091F4DC
:107B300006C085E001C084E00E94CE150BC080E243
:107B40000E94CE1585E00E94CE1580919D028F5F28
:107B500080939D0280919C028F5F80939C02833072
:107B600010F010929C021F9108950F931F93CF93D2
:107B7000DF938C010E940518EC01009731F482E03C
:107B800061E472E10E94D91718C000D000D00F92B2
:107B9000EDB7FEB7319682E0ADB7BEB711968C93C4
:107BA0008DE392E192838183D483C3830E947F1704
:107BB0000F900F900F900F900F900115110521F06D
:107BC00082E0B8010E94D917CE01DF91CF911F91B9
:107BD0000F9108950F931F93CF93DF938C010E9411
:107BE0000218EC010115110521F002301105D9F53B
:107BF00018C080E090E00E94B53D892BA1F181E0A2
:107C000060E00E9411168AA19BA1892B11F081E0EE
:107C100001C082E00E941125BC0182E00E94D917B8
:107C200022C08A819B81892BF1F488819981892BDB
:107C3000D1F08AA19BA1892BB1F081E060E00E9484
:107C4000111683E00E941125BC0182E00E94D91721
:107C500084EF91E00E9494128AA19BA10E94052CBE
:107C60001BA21AA21CA280E090E0DF91CF911F918D
:107C70000F9108950F931F93CF93DF93EB01823001
:107C8000910509F4A1C0833091053CF4009709F4F3
:107C90003EC0019709F0D4C00CC08430910509F4AE
:107CA00044C0843091050CF488C0059709F0C8C021
:107CB00061C00E940218FC0180819181892B09F426
:107CC000BFC09F012C5D3F4FAE014B5E5F4FDE0199
:107CD0001A9660E217C0F9018081882359F0E7E421
:107CE000F2E19491981721F031969923D1F702C0CF
:107CF0008C9301C06C93F9018081882311F02F5F70
:107D00003F4F1196A417B50730F31C9299C080E03D
:107D100090E00E94B53D81E060E00E9411162A9635
:107D200082E0BE010E946E178BC08981A82FB0E04F
:107D3000FB01EA0FFB1F228547E452E1FA0180E0D4
:107D40009491921731F03196992311F08F5FF8CF0B
:107D50008FEF8F5FE82FFF27E7FDF095E95BFD4E82
:107D60008491882311F4FA018491AC0FBD1F1A96F7
:107D70008C9366C08981A82FB0E0FB01EA0FFB1F3E
:107D80002285E7E4F2E180E09491921729F03196A0
:107D9000992339F08F5FF8CF882319F0E82FE1504D
:107DA00001C0EFE2FF27E7FDF095E95BFD4EE491AE
:107DB000AC0FBD1F1A96EC9343C083E090E04AE0FD
:107DC00050E00E94CA313CC00E9402188C01FC01A4
:107DD00082819381892BA1F58A81882349F489E0E6
:107DE0008B8381E0888F19821F8A8A838E8B28C0BB
:107DF00089818F5F89838F8B8B3010F11B821A8270
:107E00001E8A98012C5D3F4FD901FE013A968CE005
:107E100001900D928150E1F7F80182A193A1608158
:107E20007181009721F0458D0E948E2C06C0CB01F8
:107E3000F801658DA9010E94452DF80193A382A345
:107E400080E090E0DF91CF911F910F9108956F92A4
:107E50007F928F929F92AF92BF92DF92EF92FF92AA
:107E60000F931F93CF93DF93EC017B010E940218C5
:107E70008C01C230D10509F47EC0C330D10534F481
:107E8000209719F1219709F0E5C005C0C630D1054A
:107E90000CF0E0C031C0FC01258D922F9370848DD1
:107EA00086FF04C0992329F494E003C0992309F4C0
:107EB00091E0269526952370235083E0989FC0017A
:107EC0001124280FF7012183C5C081E060E00E94E2
:107ED00011168CED92E10E94B53D892B09F4BAC0D0
:107EE000F70161818AE0689FB001112468587D4ED6
:107EF00082E00E94D917AEC0FC01848D86FD03C0CC
:107F000049E050E002C04AE050E0CE01B7010E94D3
:107F1000CA31F801808191818F3F9105B9F0B0F0AD
:107F2000F7018181882311F486E08183F801848D33
:107F300086FD06C0F7018181863010F488E08183D8
:107F4000F7018181863010F489E08183F801808116
:107F500091818050984208F47DC0F7018181882387
:107F600011F489E08183F7018181893008F072C0C2
:107F700089E081836FC0FC0182819381892B09F0A4
:107F800069C0F7018281882309F45CC0F801608030
:107F900071806114710409F45DC0858D0E94EB1736
:107FA000EC01F7014181842F63E00E94114C292FDD
:107FB00030E0220F331F220F331F842F0E94114CF9
:107FC000D82ED394D22AF4E0DF1609F4DD24F80188
:107FD00082A093A08D2D0E94EB17F801268D422FD1
:107FE00050E04F775070BC01649FC001659F900DB9
:107FF000749F900D1124BE010E941D4C2078262BE9
:10800000268FE7012A96F4E2AF2EB12CA00EB11E06
:10801000CE01B5010E944A4CC3016D2D0E94AE4BAA
:108020008114910459F0F80160817181C401458D7A
:108030009E010E948E2CF80193A382A3C501BE016C
:108040000E944A4C90E0F7018281882309F491E074
:10805000F701928380E090E0DF91CF911F910F9123
:10806000FF90EF90DF90BF90AF909F908F907F90A8
:108070006F900895AF92BF92CF92DF92EF92FF92EE
:108080000F931F93DF93CF930F92CDB7DEB77B0192
:108090008230910509F46CC08330910534F4009767
:1080A000F1F0019709F0DFC00CC08430910509F4AC
:1080B00049C0843091050CF454C0059709F0D3C031
:1080C00047C09B01265F3F4FC90160E270E04BE073
:1080D00050E00E94434CD70155961C92C4C0FB014E
:1080E0008281882309F4BFC08181882309F4BBC041
:1080F0008B01065F1F4F90E060E070E0A8010E94D6
:108100004F2D00D000D00F92EDB7FEB7319622E090
:10811000ADB7BEB711962C932FED32E13283218398
:10812000948383830E947F170F900F900F900F907E
:108130000F9081E060E00E94111682E0B8010E9479
:108140006E1791C0FB01818190E00E948A2C05C0CE
:10815000FB01818190E00E94862CD70111968C93BF
:1081600082C083E090E040E050E00E94CA317BC0D2
:1081700090E0FB018281882309F491E0D7011296F7
:108180009C930E9402188C01F7018281882371F070
:10819000D80192968D919C919397009729F480E055
:1081A00090E00E948A2CF70181835DC0BAE0AB2E7B
:1081B000B12CAE0CBF1CD70111968C9190E0BE0182
:1081C0006F5F7F4FA5010E944F2D6C01F801848DD8
:1081D00082FF08C0C601A0E0B0E0808F918FA28F1F
:1081E000B38F3EC0D8018D919C911197009721F0DB
:1081F00015969C938E931497F8011386128613821A
:108200001282D80116961D921D921D921C921997EA
:1082100011961C921E925C968C915C978C7F5C965A
:108220008C938FEFB6010E940126F8018081918125
:10823000892B21F0C60169810E94AE4BD8018D9136
:108240009C91892B69F0C8018496B5010E944A4C23
:10825000F7018181D80192968C93929793961C9204
:108260002FEF3FEF02C020E030E0C9010F90CF9127
:10827000DF911F910F91FF90EF90DF90CF90BF9013
:10828000AF9008950F931F93CF93DF93EC018B0171
:10829000009731F097FD40C002970297E8F536C08D
:1082A00081E060E00E941116D80112968C9188231B
:1082B00059F482E065EF72E10E94D91782E06FEE17
:1082C00072E10E94D91722C00E944B25EDB7FEB77C
:1082D00037970FB6F894FEBF0FBEEDBF319622E080
:1082E000ADB7BEB711962C9323EE32E132832183D2
:1082F00063837483858396830E947F17EDB7FEB7EF
:1083000037960FB6F894FEBF0FBEEDBFCE01B80191
:1083100040E050E00E94CA3180E090E0DF91CF91D0
:108320001F910F910895CF93DF93EB018230910558
:1083300009F44AC08330910534F4009799F001970D
:1083400009F056C005C0863091050CF051C037C009
:108350000E944125DC0114968C9163E00E94114C2F
:10836000898346C081E060E00E941116998183E014
:10837000989F802D11240E948E1582E090E00E942B
:10838000941281B763E00E94114C898300D000D021
:108390000F92EDB7FEB7319692E0ADB7BEB711962A
:1083A0009C932EEF32E132832183838314820E94D7
:1083B0007F170F900F900F900F900F9019C04FEEF6
:1083C0005FEF0E94CA3114C08A81882359F00E944D
:1083D0004125298143E0249F90011124FC0124833D
:1083E0000E942C2690E08A81882309F491E09A83E8
:1083F00080E090E0DF91CF910895CF93DF93EB0180
:1084000082309105C9F1833091053CF4009751F019
:108410008130910509F058C029C0863091050CF0D3
:1084200053C024C08A81882309F44EC080E061E0F3
:108430000E9411168981845F0E94B824BC0182E0E9
:108440000E94D91781E060E00E94111669816230B4
:1084500020F08AE10E94112504C0862F805F0E94CF
:10846000B824BC0182E00E94D9172EC0BE0142E0B0
:1084700050E00E94CA3128C08A81882319F189817D
:10848000823018F48E5F89831FC081E060E00E9413
:1084900011168981833051F487E10E941125BC01B6
:1084A00082E00E94D9170E94F04509C088E10E942D
:1084B0001125BC0182E00E94D9170E94D0452FEF00
:1084C0003FEF04C081E08A8320E030E0C901DF9102
:1084D000CF910895CF92DF92EF92FF920F931F9367
:1084E000CF93DF937C01162F0E9405160E94412531
:1084F0006C01173208F06AC0C12FD0E08E01000F66
:10850000111F000F111F0C0F1D1F0D5E1E4FD701F5
:1085100012968C91882311F080E001C081E00E94C6
:10852000CE15F6018581843059F0853089F0BE0181
:1085300024E0660F771F2A95E1F78130B1F412C06D
:1085400094E0CC0FDD1F9A95E1F7C45FDC4E07C0C5
:1085500084E0CC0FDD1F8A95E1F7C458DA4E82E043
:10856000BE0106C06452784E02C0645C754E82E063
:108570000E94D917D70112968C91882389F4F801AB
:10858000848187FD0DC081E060E00E941116D80152
:1085900014968C910E941125BC0182E00E94D9178B
:1085A000D8011296ED91FC911397309721F080E05D
:1085B00090E0B7010995F7018689882329F0808D1D
:1085C00067890E94B51602C00E940D16DF91CF91F7
:1085D0001F910F91FF90EF90DF90CF9008952F9211
:1085E0003F924F925F926F927F928F929F92AF9243
:1085F000BF92CF92DF92EF92FF920F931F93DF9380
:10860000CF93CDB7DEB76B970FB6F894DEBF0FBE32
:10861000CDBFD82E45E2481708F45CC2DE011196A2
:108620008BE1FD0111928A95E9F7A8958D2D90E0D7
:10863000FC01EE0FFF1FEE0FFF1FE80FF91FED5EAD
:10864000FE4F0280F381E02D309721F081E090E031
:10865000BD0109958E010F5F1F4FC8016D2D0E944E
:108660006A420E9402184C0158018EEF682E8FEF6B
:10867000782E0FEF402E0FE7502E1BE0212E312CCD
:108680002C0E3D1EF5E0DF9E80011124B3E1EB2EA0
:10869000B1E0FB2EE00EF11E0E947D0E0E946514DB
:1086A0009C018B30910509F4D1C08C3091058CF47C
:1086B0008A3091050CF02DC1813091050CF04BC131
:1086C0004FEF8F3F940709F4F6C1009709F433C1C7
:1086D000E3CF8731910509F4B9C08831910544F49D
:1086E0008531910509F4CAC186319105A9F6CFC13A
:1086F0008A31910509F450C08232910509F4E5C12F
:108700008931910549F68B81882369F0D70112964A
:10871000ED91FC911397309719F084E090E0ABC194
:108720008A818F5F48C01F8AF801ED5EFE4F10817D
:10873000A5E0EA2EF12CEE0EFF1ED3940E94021843
:10874000FC01848D86FD0AC0F2E0DF1639F485E075
:1087500090E0E80EF91EF3E0DF2E03C095E29D15D0
:108760002CF0D7018C91811709F45EC0A3E1B1E030
:1087700060E0E12FFF27E7FDF0958C9190E08E17E8
:108780009F0711F4D62E50C06F5F663211F0159618
:10879000F4CFDD24DA9448C08B81882371F0D701AF
:1087A0001296ED91FC911397309719F085E090E0C7
:1087B00062C18A8181508A8388C11F8A0D5E1E4FE3
:1087C000F801C080EBEFEE2EEFEFFE2EE00EF11E73
:1087D000DA940E940218DC015C968C9186FD0BC035
:1087E000B2E0DB1641F47801E6EFFFEFEE0EFF1E7C
:1087F000DD24D39402C0D7FC04C0D7018C918C1522
:1088000099F0ECECF1E075E2D72E2C2D332727FD03
:108810003095808190E08217930731F0DA94BFEFB2
:10882000DB1611F03597F5CF8D2D90E0FC01EE0FA2
:10883000FF1FEE0FFF1FE80FF91FED5EFE4F0280D6
:10884000F381E02D309709F05AC03FC1F7019181C3
:108850009923E9F1A92FB0E0FD01E256FD4F808197
:108860001816BCF0E3E1F1E020E0492F552747FD61
:108870005095808190E08417950711F4822F06C0EF
:108880002F5F263211F03596F4CF8FEFA256BD4FF1
:108890008C93D7011196EC91F0E0E256FD4F808168
:1088A0000E94EF42282F332727FD3095F701818161
:1088B000E82FF0E0E256FD4FC90137FF04C08827DA
:1088C0009927821B930B808337FFFFC00DC0D70110
:1088D0001296ED91FC9113973097A1F082E090E011
:1088E000B501099597FF02C0D194F5C08B8188230B
:1088F00009F0EBC0D7011296ED91FC91139781E03E
:1089000090E0B9C090E08B81882309F491E09B83CB
:10891000DCC08B81882309F4DEC0D7011296ED916B
:10892000FC911397309729F083E090E0B501099509
:10893000DDCF1B82CAC08C81813009F4A3CE883080
:1089400051F481E00E9466488A810E94AE4880E02E
:108950000E946648BAC08C81853009F461C08630B7
:1089600070F4823041F1833020F4813009F0ADC0E1
:1089700012C0833081F0843009F0A7C04EC0873028
:1089800009F463C0873008F45AC0883021F0893078
:1089900009F09BC060C08F819885892B11F458869F
:1089A0004F828F819885821793070CF48EC01E82A8
:1089B0001D8282E08C838D819E818C0153E0000FAB
:1089C000111F5A95E1F7880F991F080F191F020F01
:1089D000131FF401848D86FD15C0F7E7013A1F07C8
:1089E00089F482E00E94824B81E060E00E941116CF
:1089F00082E068E971E10E94D91784EF91E00E945A
:108A0000941202C017FD61C08F819885801791076D
:108A10000CF45BC01E830D8358C0198645E04C835F
:108A20008985AAE08A9FC0011124820F931F8F3F7E
:108A3000910509F008F489877B8E6A8E46C028303C
:108A400031050CF042C02A8740C022303105ECF5D8
:108A50003B8F2A8F3AC08A81F101E80FF11D822FE6
:108A6000805D8083D7011296ED91FC91139730972A
:108A700061F182E090E0B501099527C080E00E9495
:108A80004A0F80E060E240E00E9420271EC0D7012C
:108A90001296ED91FC911397309721F086E090E0CB
:108AA000B5010995F7018081882379F483E290E08C
:108AB0000E944B2010C08C81883009F0E3CD80E00B
:108AC00090E0B5010E94B03CDDCDC5016D2D0E9446
:108AD0006A42D8CDDD248D2D6B960FB6F894DEBF9B
:108AE0000FBECDBFCF91DF911F910F91FF90EF90FF
:108AF000DF90CF90BF90AF909F908F907F906F90BE
:108B00005F904F903F902F9008951F93182F0E94D1
:108B10005925803809F442C080E060E372E00E9489
:108B2000F21681E068E272E00E94F21680919E02E5
:108B3000863210F010929E0217FD04C0812F0E9411
:108B4000EF420EC080919E020E94EF42992787FD5E
:108B5000909597FF03C0909581959F4F80939E02BB
:108B600080E06CE171E00E94F21681E060E671E065
:108B70000E94F21684E068E871E00E94F21685E037
:108B800060E971E00E94F21686E068E971E00E94F7
:108B9000F21687E060EA71E00E94F2161F910895D4
:108BA000DF93CF9300D000D000D0CDB7DEB7FE0169
:108BB000319686E0DF011D928A95E9F788E0898386
:108BC0001A8284E2BF014DE959E40E949E2726964D
:108BD0000FB6F894DEBF0FBECDBFCF91DF910895E1
:108BE000DF93CF9300D000D000D0CDB7DEB7FE0129
:108BF000319686E0DF011D928A95E9F788E0898346
:108C000081E08A8384E2BF014DE959E40E949E27F6
:108C100026960FB6F894DEBF0FBECDBFCF91DF9181
:108C20000895DF92EF92FF920F931F93DF93CF93FC
:108C300000D000D000D0CDB7DEB7D82E8E010F5FA8
:108C40001F4F86E0F80111928A95E9F782E0898347
:108C50001A8287E08B838DEAE82E89E4F82E84E27D
:108C6000B801A7010E949E2781E089831A82DB82D6
:108C700084E2B801A7010E949E2726960FB6F894B9
:108C8000DEBF0FBECDBFCF91DF911F910F91FF903F
:108C9000EF90DF900895DF93CF9300D000D000D005
:108CA000CDB7DEB7FE01319686E0DF011D928A95D1
:108CB000E9F7198284E2BF014DEA59E40E949E2738
:108CC00026960FB6F894DEBF0FBECDBFCF91DF91D1
:108CD00008950F93DF93CF9300D000D000D0CDB78D
:108CE000DEB7542F46E14983482F4F774A83880FD8
:108CF000892F881F990B91958F778B83822F8F7780
:108D00008C83220F232F221F330B319527702D8345
:108D1000802F8F778E8307FF02C028602D83862FD8
:108D200090E08370907024E0880F991F2A95E1F7F6
:108D30009D81982B9D83552311F090649D8384E23F
:108D4000BE016F5F7F4F4DEB59E40E949E27269630
:108D50000FB6F894DEBF0FBECDBFCF91DF910F915C
:108D60000895DF93CF9300D000D000D0CDB7DEB709
:108D7000FE01319696E0DF011D929A95E9F794E1A4
:108D80009983982F9F779A83881F8827881F8B83C2
:108D900084E2BF014DEB59E40E949E2726960FB650
:108DA000F894DEBF0FBECDBFCF91DF910895DF9362
:108DB000CF9300D000D000D0CDB7DEB7FE01319602
:108DC00096E0DF011D929A95E9F78983862F8F77C8
:108DD0008A83660F672F661F770B71956F776B839A
:108DE000842F8F778C83441F4427441F4D8384E254
:108DF000BF014DEB59E40E949E2726960FB6F894CA
:108E0000DEBF0FBECDBFCF91DF9108959C01462FED
:108E100083E1B9010E94D74608959C01462F8DE059
:108E2000B9010E94D7460895DF93CF9300D000D0B8
:108E300000D0CDB7DEB7FE01319696E0DF011D927E
:108E40009A95E9F78983862F8F778A83660F672F34
:108E5000661F770B71956F776B8384E2BF014DEBD3
:108E600059E40E949E2726960FB6F894DEBF0FBEE7
:108E7000CDBFCF91DF910895BC0182E10E941447DC
:108E80000895BC018CE00E9414470895DF93CF93AE
:108E900000D000D000D0CDB7DEB7FE01319696E00D
:108EA000DF011D929A95E9F791E199838F708A838A
:108EB000862F8F778B83661F6627661F6C8384E2FD
:108EC000BF014DEB59E40E949E2726960FB6F894F9
:108ED000DEBF0FBECDBFCF91DF910895DF93CF935B
:108EE00000D000D000D0CDB7DEB7FE01319696E0BD
:108EF000DF011D929A95E9F790E199838F708A833B
:108F000084E2BF014DEB59E40E949E2726960FB6DE
:108F1000F894DEBF0FBECDBFCF91DF910895DF93F0
:108F2000CF9300D000D000D0CDB7DEB7FE01319690
:108F300026E0DF011D922A95E9F72FE02983282FEB
:108F40002F772A83880F892F881F990B91958F7708
:108F50008B8367706C831D82442311F081E08D83C5
:108F600084E2BE016F5F7F4F4DEB59E40E949E2764
:108F700026960FB6F894DEBF0FBECDBFCF91DF911E
:108F80000895DF93CF9300D000D000D0CDB7DEB7E7
:108F9000FE01319626E0DF011D922A95E9F72EE0C9
:108FA0002983282F2F772A83880F892F881F990BD1
:108FB00091958F778B8367706C8384E2BF014DEB53
:108FC00059E40E949E2726960FB6F894DEBF0FBE86
:108FD000CDBFCF91DF910895DF93CF9300D000D024
:108FE00000D0CDB7DEB7FE01319696E0DF011D92CD
:108FF0009A95E9F797E099839FE79A839B838F7708
:109000008C8384E2BF014FED59E40E949E2726968F
:109010000FB6F894DEBF0FBECDBFCF91DF9108959C
:10902000DF93CF9300D000D000D0CDB7DEB7FE01E4
:10903000319626E0DF011D922A95E9F727E0298382
:10904000282F2F772A83880F892F881F990B9195B6
:109050008F778B836F776C8384E2BF014FED59E488
:109060000E949E2726960FB6F894DEBF0FBECDBF96
:10907000CF91DF910895DF93CF9300D000D000D03F
:10908000CDB7DEB7FE01319626E0DF011D922A95AD
:10909000E9F727E02983282F2F772A83880F892F44
:1090A000881F990B91958F778B838FE78C8384E250
:1090B000BF014FED59E40E949E2726960FB6F89403
:1090C000DEBF0FBECDBFCF91DF910895DF93CF9369
:1090D00000D000D000D0CDB7DEB7FE01319696E0CB
:1090E000DF011D929A95E9F7882311F482E001C00F
:1090F00081E0898380E48A8384E2BE016F5F7F4FD1
:109100004FEE59E40E949E2726960FB6F894DEBFD4
:109110000FBECDBFCF91DF910895DF93CF9300D0E5
:1091200000D000D0CDB7DEB796E0FE013196DF016A
:10913000292F1D922A95E9F799838F778A8384E2F4
:10914000BF014FEF59E40E949E2726960FB6F89470
:10915000DEBF0FBECDBFCF91DF910895DF93CF93D8
:1091600000D000D000D0CDB7DEB7FE01319696E03A
:10917000DF011D929A95E9F795E099838F778A83AD
:1091800084E2BF014FEF59E40E949E2726960FB656
:10919000F894DEBF0FBECDBFCF91DF910895DF936E
:1091A000CF9300D000D000D0CDB7DEB7FE0131960E
:1091B00096E0DF011D929A95E9F794E099838F7705
:1091C0008A8384E2BF0145E25AE40E949E272696E4
:1091D0000FB6F894DEBF0FBECDBFCF91DF910895DB
:1091E000DF93CF9300D000D000D0CDB7DEB7FE0123
:1091F000319686E0DF011D928A95E9F784E0898344
:109200008FE78A8384E2BF0145E25AE40E949E27E9
:1092100026960FB6F894DEBF0FBECDBFCF91DF917B
:109220000895DF93CF9300D000D000D0CDB7DEB744
:10923000FE01319696E0DF011D929A95E9F793E0E1
:10924000998391E09A83982F9F779B83881F882723
:10925000881F8C8384E2BF0145E35AE40E949E2765
:1092600026960FB6F894DEBF0FBECDBFCF91DF912B
:109270000895DF93CF9300D000D000D0CDB7DEB7F4
:10928000FE01319686E0DF011D928A95E9F783E0C1
:1092900089831A8284E2BF0145E35AE40E949E2733
:1092A00026960FB6F894DEBF0FBECDBFCF91DF91EB
:1092B0000895DF93CF9300D000D000D0CDB7DEB7B4
:1092C00084E068EF71E00E94F21685E060E072E0F1
:1092D0000E94F21687E79DE368EC70E00E94561545
:1092E000FE01319686E0DF011D928A95E9F78BE059
:1092F000898384E2BF014DE859E40E949E27892BAF
:1093000019F40E947D0EFDCF26960FB6F894DEBFAD
:109310000FBECDBFCF91DF910895FC0181818432D2
:1093200019F482818B3021F0CF010E94C826089564
:1093300080E090E00E94FE2B0895FC018181843240
:1093400019F48281883021F0CF010E94C826089547
:1093500080E090E00E94FE2B0895FC018181843220
:1093600019F48281882321F0CF010E94C826089534
:10937000848190E00E94FE2B0895FC01818184325B
:1093800019F48281853121F0CF010E94C826089509
:10939000438150E0848190E09695982F8827979597
:1093A00087956581362F3295330F330F307C20E05F
:1093B000822B932B842B952B0E94FE2B0895FC016E
:1093C0008181843219F48281873021F0CF010E949B
:1093D000C8260895858190E00E94FE2B0895FC0127
:1093E0008181843219F48281882321F0CF010E9487
:1093F000C8260895838190E00E94FE2B0895FC0109
:109400008181843219F48281853021F0CF010E945C
:10941000C8260895238130E02F7730704581942F3E
:109420009295990F990F907C80E0822B932B248149
:1094300030E02F7730703695322F222737952795D9
:10944000822B932B0E94FE2B0895FC018181843294
:1094500019F48281843021F0CF010E94C82608953A
:10946000838190E00E94FE2B0895FC01818184326B
:1094700019F48281833021F0CF010E94C82608951B
:109480008481881F8827881F9381892B90E00E9400
:10949000FE2B0895DF93CF93CDB7DEB72A970FB693
:1094A000F894DEBF0FBECDBFFE01359626E0DF018A
:1094B0001D922A95E9F729E02D83282F2F772E83F7
:1094C000880F892F881F990B91958F778F8384E25E
:1094D000BF0146E85AE49E012F5F3F4F0E943B27A1
:1094E000892B29F020E030E040E050E004C02981E1
:1094F0003A814B815C81B901CA012A960FB6F89472
:10950000DEBF0FBECDBFCF91DF910895DF93CF9324
:1095100000D000D0CDB7DEB7FC018181843229F4C0
:109520006281862F8950823020F0CF010E94C826A8
:1095300082C0838190E0A0E0B0E0248130E040E090
:1095400050E077E0220F331F441F551F7A95D1F763
:10955000282B392B4A2B5B2B858190E0A0E0B0E0D3
:109560007EE0880F991FAA1FBB1F7A95D1F7282B81
:10957000392B4A2B5B2B868190E0A0E0B0E075E1AF
:10958000880F991FAA1FBB1F7A95D1F7282B392B5B
:109590004A2B5B2B878190E0A0E0B0E07CE1880F54
:1095A000991FAA1FBB1F7A95D1F7282B392B4A2B5D
:1095B0005B2B29833A834B835C836A3059F581E0C6
:1095C00060E00E9411168DB79EB707970FB6F8940A
:1095D0009EBF0FBE8DBFEDB7FEB7319682E0ADB72F
:1095E000BEB711968C938CE99CE19283818389812B
:1095F0009A81AB81BC8183839483A583B6830E94C7
:109600007F178DB79EB707960FB6F8949EBF0FBE13
:109610008DBF11C0211531054105510519F080E0BC
:1096200090E002C08FEF9FEFBE016F5F7F4F44E07D
:1096300050E00E94E62B0F900F900F900F90CF916B
:10964000DF9108951F93DF93CF9300D000D000D017
:10965000CDB7DEB7182F813021F0843011F088307B
:10966000B9F4FE01319686E0DF011D928A95E9F793
:10967000198284E2BF014FEE59E40E949E2740E028
:10968000212F30E028233923232B29F041E003C088
:109690000E944425482F842F26960FB6F894DEBFEB
:1096A0000FBECDBFCF91DF911F910895DF93CF9370
:1096B00000D000D000D0CDB7DEB7982F813031F088
:1096C000843021F0883011F0823089F4FE01319627
:1096D00086E0DF011D928A95E9F782E089839A830B
:1096E00084E2BF014FEE59E40E949E2702C00E940F
:1096F000442626960FB6F894DEBF0FBECDBFCF919D
:10970000DF910895DF93CF9300D000D000D0CDB784
:10971000DEB7982F813031F0843021F0883011F09D
:10972000823089F4FE01319686E0DF011D928A9530
:10973000E9F781E089839A8384E2BF014FEE59E41F
:109740000E949E2702C00E944D2626960FB6F894CE
:10975000DEBF0FBECDBFCF91DF9108950F931F9352
:10976000DF93CF9300D000D000D0CDB7DEB78C010F
:10977000FE01319686E0DF011D928A95E9F7802F80
:109780008F778983C801880F892F881F990B91953E
:109790008F778A836F776B838FEF64E0AF010E94CE
:1097A0000A2781E060E00E94111680E00E941125E6
:1097B000BC0182E00E94D91780E090E060E040E0C8
:1097C00050E00E94F91A8FEFB8010E9401262696F8
:1097D0000FB6F894DEBF0FBECDBFCF91DF911F91C2
:1097E0000F910895629FD001739FF001829FE00D59
:1097F000F11D649FE00DF11D929FF00D839FF00D10
:10980000749FF00D659FF00D9927729FB00DE11DBB
:10981000F91F639FB00DE11DF91FBD01CF01112498
:109820000895991B79E004C0991F961708F0961BBC
:10983000881F7A95C9F780950895AA1BBB1B51E133
:1098400007C0AA1FBB1FA617B70710F0A61BB70BB0
:10985000881F991F5A95A9F780959095BC01CD0155
:109860000895FC0105900020E9F7809590958E0FF2
:109870009F1F0895FB01DC0102C001900D92415031
:109880005040D8F70895DC0101C06D93415050401D
:10989000E0F70895FB01DC0101900D920020E1F753
:1098A00008950F931F93DF93CF93CDB7DEB72E9715
:1098B0000FB6F894DEBF0FBECDBF8C0186E08C835F
:1098C0001A8309838FEF9FE79E838D83CE010196D4
:1098D0000E94A34CEF81F885E00FF11F10822E96B5
:1098E0000FB6F894DEBF0FBECDBFCF91DF911F91B1
:1098F0000F9108950F931F93DF93CF93CDB7DEB7EA
:109900002E970FB6F894DEBF0FBECDBF8C018EE050
:109910008C831A8309838FEF9FE79E838D83CE010B
:1099200001960E94A34CEF81F885E00FF11F108291
:109930002E960FB6F894DEBF0FBECDBFCF91DF914C
:109940001F910F9108952F923F924F925F926F92C5
:109950007F928F929F92AF92BF92CF92DF92EF92BF
:10996000FF920F931F93DF93CF93CDB7DEB72B9763
:109970000FB6F894DEBF0FBECDBF3C012B015A01DC
:10998000FC0117821682838181FD03C06FEF7FEF98
:10999000C6C19AE0892E1E010894211C311CF301D6
:1099A0002381F20123FD859123FF81912F018823DB
:1099B00009F4B2C1853239F423FD859123FF8191E9
:1099C0002F01853229F490E0B3010E94E44EE7CFE5
:1099D000982FFF24EE249924FFE1FF15D0F09B324D
:1099E00069F09C3228F4903259F0933291F40EC011
:1099F0009D3249F0903369F441E024C052E0F52AE9
:109A000084E0F82A28C098E0F92A25C0E0E1FE2A7F
:109A100022C0F7FC29C0892F80538A3070F4F6FEEB
:109A200005C0989C902C1124980E15C0E89CE02C41
:109A30001124E80EF0E2FF2A0EC09E3229F4F6FC53
:109A40006BC140E4F42A07C09C3619F450E8F52AAB
:109A500002C0983649F4F20123FD959123FF9191BC
:109A60002F01992309F0B8CF892F8554833018F03E
:109A70008052833038F444E050E0A40EB51E5FE31A
:109A800059830FC0933631F0933779F0933509F04D
:109A900056C020C0F5018081898342E050E0A40EC9
:109AA000B51E610101E010E012C0F501C080D18057
:109AB000F6FC03C06FEF7FEF02C0692D70E042E05B
:109AC00050E0A40EB51EC6010E94D94E8C015FE77E
:109AD000F52214C0F501C080D180F6FC03C06FEF01
:109AE0007FEF02C0692D70E042E050E0A40EB51E89
:109AF000C6010E94CE4E8C0150E8F52AF3FE07C045
:109B00001AC080E290E0B3010E94E44EEA948E2DE8
:109B100090E008171907A8F30EC0F601F7FC85912D
:109B2000F7FE81916F0190E0B3010E94E44EE110D5
:109B3000EA94015010400115110579F7EAC09436F6
:109B400011F0993669F5F7FE08C0F50120813181E1
:109B50004281538184E090E00AC0F50180819181C7
:109B60009C01442737FD4095542F82E090E0A80ED9
:109B7000B91E9FE6F92257FF09C0509540953095D0
:109B800021953F4F4F4F5F4FE0E8FE2ACA01B901D0
:109B9000A1012AE030E00E94104FD82ED21840C018
:109BA000953729F41F2D1F7E2AE030E01DC01F2DA0
:109BB000197F9F3661F0903720F4983509F0ACC0DA
:109BC0000FC0903739F0983709F0A6C004C028E0DC
:109BD00030E00AC0106114FD146020E130E004C0E0
:109BE00014FD166020E132E017FF08C0F501608126
:109BF00071818281938144E050E008C0F501808149
:109C00009181BC0180E090E042E050E0A40EB51EDE
:109C1000A1010E94104FD82ED2188FE7F82EF12202
:109C2000F6FE0BC05EEFF522D91438F4F4FE07C03F
:109C3000F2FC05C08FEEF82202C01D2D01C0192DC7
:109C4000F4FE0DC0FE01ED0DF11D8081803319F48D
:109C500099EEF92208C01F5FF2FE05C003C08F2DE8
:109C6000867809F01F5F0F2DF3FC14C0F0FE0FC0C3
:109C70001E1510F09D2C0BC09D2C9E0C911A1E2DB4
:109C800006C080E290E0B3010E94E44E1F5F1E1503
:109C9000C0F304C01E1510F4E11A01C0EE2404FF45
:109CA0000FC080E390E0B3010E94E44E02FF1DC0AC
:109CB00001FD03C088E790E00EC088E590E00BC08E
:109CC000802F867891F001FF02C08BE201C080E214
:109CD000F7FC8DE290E0B3010E94E44E06C080E301
:109CE00090E0B3010E94E44E9A94D914C0F3DA9440
:109CF000F101ED0DF11D808190E0B3010E94E44E71
:109D0000DD20A9F706C080E290E0B3010E94E44E96
:109D1000EA94EE20C1F743CEF30166817781CB014F
:109D20002B960FB6F894DEBF0FBECDBFCF91DF915B
:109D30001F910F91FF90EF90DF90CF90BF90AF9069
:109D40009F908F907F906F905F904F903F902F905B
:109D50000895DC01CB01FC01E199FECF06C0FFBBF9
:109D6000EEBBE09A31960DB20D9241505040B8F7DB
:109D70000895E199FECF9FBB8EBBE09A99278DB3E2
:109D80000895262FE199FECF9FBB8EBB2DBB0FB64A
:109D9000F894E29AE19A0FBE01960895FC010590AD
:109DA000615070400110D8F7809590958E0F9F1FDD
:109DB0000895FC016150704001900110D8F7809522
:109DC00090958E0F9F1F08950F931F93CF93DF934E
:109DD0008C01EB018B8181FF1BC082FF0DC02E81A6
:109DE0003F818C819D812817390764F4E881F981CE
:109DF0000193F983E88306C0E885F985802F0995EA
:109E0000892B31F48E819F8101969F838E8302C0BE
:109E10000FEF1FEFC801DF91CF911F910F910895B0
:109E2000FA01AA27283051F1203181F1E8946F938B
:109E30006E7F6E5F7F4F8F4F9F4FAF4FB1E03ED031
:109E4000B4E03CD0670F781F891F9A1FA11D680FCF
:109E5000791F8A1F911DA11D6A0F711D811D911D02
:109E6000A11D20D009F468943F912AE0269F112477
:109E70003019305D3193DEF6CF010895462F4770DB
:109E8000405D4193B3E00FD0C9F7F6CF462F4F7036
:109E9000405D4A3318F0495D31FD4052419302D094
:109EA000A9F7EACFB4E0A69597958795779567953A
:109EB000BA95C9F700976105710508959B01AC013A
:109EC0000A2E06945795479537952795BA95C9F761
:109ED000620F731F841F951FA01D0895F894FFCF74
:109EE000FFFFFFE9282534642D2534643A2000253E
:109EF00034640000010000FF00020000FF000700C2
:109F000000FF0000FD41FF00030000FF000093413F
:109F1000FF00004241FF00000B32FF01003A40FF0A
:109F20000100273FFF01003A3EFF0100EA3DFF022A
:109F300000783AFF0200103CFF0200A03BFF020045
:109F4000B13AFF0200643AFF0200503AFF02001CDF
:109F50003AFF02004638FF0300ED34FF03008C3463
:109F6000FF03040000FF0300BC371B0305000022B1
:109F7000030600002203000337FF0300FE36FF0341
:109F8000006537FF04000837FF0400B03CFF050000
:109F9000F936FF05004D36FF0600FE35FF06003896
:109FA00035FF06008834FF06008434FF0700FB32CB
:029FB000FF00B0
:00000001FF
